:020000041100E9
:10300000002373B52B4D2C4C28006361022601F080
:103010005DFA4021FE2221742800284B009601F021
:10302000A7FA002836D1217CFF222800244B0096E5
:1030300001F09EFA00282DD1224BA2899A4226D176
:10304000E389214A93420DD1204B6361204B2268D2
:10305000002A03D1002B01D043CB43C4280001F048
:1030600073FA73BD1B4A934201D00023EFE71A4B5A
:103070001A4A1B68934206D9C02304222800217CE7
:103080009B0001F0EBFA114B6361154BDFE7002366
:103090002374EAE7CC233821AC2228009B01217459
:1030A00001F0DCFA0028F2D10E4B63610E4BE38194
:1030B0000E4BCCE7E444FF1F9064FF1F9C64FF1F8E
:1030C0009E64FF1F5959000083050000F94200115A
:1030D00038BF001182150000B464FF1F8713000081
:1030E00044BF0011B1430011AAAAFFFF2CBF001179
:1030F000F7B5164B0192C318021D002000938823D8
:103100005B05D3181B685C1C1AD09CB2402C18D8E5
:103110008D781E0CAC466746CD782D023D43AE42FD
:1031200006D1019800280ED110000C70240A4C70B2
:1031300003249BB20733A343D218009B9A42DED3E9
:10314000FEBD4432F9E71000FAE7C046FC0F00006C
:10315000802213B503000324019189B25201073183
:103160009B18A14304305A1A88235B05C3181B68B7
:10317000591C03D190429241104016BD99B240298A
:1031800007D80B000733A343C0189042ECD30020AC
:10319000F3E74430F9E7134B134A1B68126810B584
:1031A000FA24934201D81A00F824104BE4021B6859
:1031B0009A4210D813000E4A12689A420ED3013375
:1031C00007D1F823DB029C4203D10A49054808F0E5
:1031D00047FB200010BDFC24E402ECE7FE24E402DF
:1031E000F7E7C04600C0071100D0071100E0071143
:1031F00000F00711FFFFFF7FF0B59BB015000490B2
:103200000391402A00D9A0E006AB59801A80FFF74D
:10321000C2FF0400042816D9002206A9FFF768FFA0
:10322000052810D906AB1B88AB420CD1002D07D066
:10323000514B2A000499C01808F0B2FD002802D1B1
:1032400001201BB0F0BD06AB1D8020000699FFF7E2
:103250007FFF041E7BD1069B0793FFF79CFF802313
:103260005B01C618802307001B039E4201D3F8268A
:10327000F60288235B05F31801931B68013302D023
:10328000019808F0CDFC3D49019808F0E9FA3B1D92
:103290000293331D05938822029B52059B181B68DD
:1032A00008935A1C3CD044219AB20091402A04D879
:1032B0000320D11D814389B2009103991B0C8B42DD
:1032C00024D0402A22D80122300008A9FFF710FF9D
:1032D000021E1BD1380008A9FFF70AFF04000428CA
:1032E00031D9009A059B9B1880225201B218934253
:1032F00040D288235B05C118009A09A808F010FB8A
:103300001D4B009A09A9F01808F0E2FC009A029BF4
:103310009446634402931A4B029AFB189A42BAD31A
:1033200088235B05FC1821680198013908F098FA98
:10333000200008F075FC039A07AB5A80300007990B
:10334000FFF706FF0400002C03D1002079E70428D2
:10335000FBD988235B05E018069908F081FA03235E
:10336000EA1C9A4300D16BE7034B0499E01808F07C
:10337000AFFC65E70424ECE704000011FFFFFF7FCA
:10338000F80F0000F7B505001400402A21D80027E7
:1033900001AE71803780FFF7FEFE042816D93A008F
:1033A0003100FFF7A5FE042810D93688BC420BD0A7
:1033B000BD4209D0221CB44200D9321C064B92B245
:1033C000C118280008F0ACFA30B2FEBDC04300B20C
:1033D000FBE703204042F8E70400001137B5042260
:1033E00004000D0001A81649FFF7CCFF02000428D5
:1033F0000BD1019BA34208D3AB4204D0104901A8D2
:103400000195FFF7F9FE01203EBD0E4C2368200018
:10341000019308F005FC019920000139019108F0A1
:103420001FFA80235B01E418074B9C42EED1042273
:10343000034901A80195FFF7DFFE0020E4E7C0463D
:103440005555000000C007110000081130B589B0C3
:1034500008F09EFC10226946254808F0B9FB254B70
:10346000009A9A420ED1019B029A0F2B33D8002169
:1034700001240698013B08D2002900D00292029B49
:10348000013331D10023029325E0551CF2D1020013
:103490002100EFE710341022200004A908F098FB67
:1034A000029B013301D1069B0293882304995B059B
:1034B000C918059B06981A03120B049105928142C4
:1034C00003D02B4201D108F02BFA019B013B019361
:1034D000019B002BDED1029B002B03D004930498A8
:1034E0004168084709B030BDE025014C2D03EFE7E6
:1034F0000000011150485936F7B50F4F0F4BFA6DC8
:1035000004001A4084235B001343FB65030010335F
:10351000019300252E00112008F0FAF90322BB6E5A
:103520001340AB4002351E43202DF4D1019B40C413
:10353000A342EED1F7BDC04600F0004000FEFEFF02
:10354000802270B5AD4CAE4BD200002120001C6033
:1035500008F0CEFA2300AB4A88331A60AA4B1A78D7
:103560006E23002A00D01133E3620A232365A74BA0
:103570001878A74BA0630138E361C3B2032B01D8CD
:1035800010232362A34B37226361C823DB00A361AE
:1035900023008C331A60082336210F3AE518E163C3
:1035A00023646264E9670439251DE96725003B2629
:1035B000BC352E602500C0352B602500C4352A603F
:1035C00025000636CC352E602500083EC8352E6015
:1035D0002500D03529602100D4310B602100D8317D
:1035E0000A6021000225E0310D6025004221DC3512
:1035F000296025001B3EE4352E602500E8352B6050
:103600002500EC352A6022000525F43215602200E1
:10361000F032116022001831903211602200943291
:10362000136023003C2298331A60AF23DB00236031
:10363000794B2363032805D808F0D2FA33023537D3
:103640001523636096232100FA225B00A360E360E8
:10365000C8332361714BFC319200A3640A6062623B
:103660006F4A704DA2627322E2656D3A6265A2658F
:103670000232E5644A600221616696218900A166F2
:10368000626709210022E166A2676749674A684EBE
:103690002167E2673560032811D808F0A1FA96087F
:1036A0009EA61023CDE70E23CBE70C23C9E720000D
:1036B0001A259C30056020000735A03005602000E9
:1036C000A83003602300FA20F8338000186023003C
:1036D0006420A433186023005F38AC3318602300E3
:1036E0000338B03318602300C630B43318602300A9
:1036F0000020B833186023003825FC339D604D4D01
:103700005A665D644C4D9A64DD619625AD001D627C
:103710004A4D9A675D62F53DFF3D9D621E25484A10
:10372000DD6618675867D9651966DA67BE23C02158
:10373000444A5B00E250444B4900635004316250FC
:10374000C4225200A350FA23E4205B000432A350A9
:103750000432A3503D493E4A3E4BD1603E49800071
:1037600019503E49E938FF3819503D490430195085
:103770003C491038D1613C4911633C4951633C4993
:1037800011603C49195019003B48F83108603B4929
:10379000D16582213A4A89005A501A0039490832C3
:1037A000D1671A003849B43211608821374A89003C
:1037B0005A501A00364988321160364ADA6408F0E5
:1037C0009FF9012008F094FA70BD200014259C3068
:1037D000056020000435A03070E7200010259C30E3
:1037E000056020000335A03068E720000E259C30DE
:1037F000056020000235A03060E7C0460004FF1FCE
:103800006C67FF1F6072FF1F2447FF1F4A0AFF1FDC
:103810003A07000080C3C9019A02000050C30000AB
:103820006A180000280A0000204E000088130000DB
:10383000F009FF1F001F001168100000C4090000FC
:10384000DC05000040420F0010270000FD1BFF1F99
:10385000FC00FF1F0000FF1F012FFF1F2932FF1F69
:10386000C130FF1FD51FFF1FF11FFF1F9D21FF1F2D
:10387000491FFF1FC128FF1F692CFF1FD918FF1FF9
:10388000CD27FF1F3525FF1F4125FF1F491EFF1FA5
:10389000011FFF1FC11DFF1FF7B50B0CFF270122E2
:1038A000009300233C001E001D009446019089B245
:1038B00062469A401000084018413618B6B2FF2FF1
:1038C00002D1012E00D19FB2009802401A41AD18DA
:1038D000ADB2FF2C02D1012D00D19CB20133102BCF
:1038E000E6D10320012E07D1012D04D1019B240133
:1038F000E4191C700138FEBD102EFCD10238102DC9
:10390000F9D00230F7E710B5064C2378002B07D129
:103910000548FFF7F1FD0548FFF7EEFD0123237091
:1039200010BDC0462D67FF1F4067FF1F3067FF1F98
:10393000F0B58BB00D0001230190102936D8FFF7A8
:10394000E2FF00231A001B48C15C01335218102B00
:10395000FAD1023B002A29D0174B184C1F680023CC
:1039600006A9E25C1600FA5C56405E540133102B47
:10397000F7D102AA08F0B4F92A0002A9019808F0C8
:103980006FF908F04DFA23681B18236008F048FA15
:1039900063681B18636008F043FAA3681B18A360F0
:1039A00008F03EFAE3681B18E360002318000BB030
:1039B000F0BDC0464067FF1FC445FF1F3067FF1FB3
:1039C0000223F0B501245C4D5C4E2B705C4B91B032
:1039D0001C705C4F039333682000BB7006F0C6FC7C
:1039E0000023984205D0BA78552A02D0332A00D055
:1039F00096E03360002006F027FF07F099FFFFF7FD
:103A00009FFD07F0D5FF1F22012400214E4B3626D3
:103A10001A704E4B1C704E4B19704E4B19689143E7
:103A2000163A0A431A60602219689143403A0A43E1
:103A30001A6008F065F908F043F9C120FF21464BF0
:103A400080001A588A431A50C52292009858884319
:103A5000BF39014399509858404908408021C90115
:103A60000143802099509958C0050902090A014371
:103A7000995080213A48490108F01AF9032322009D
:103A8000009338490194384808F0E2F82E2237496B
:103A900004A807F045FF02AB04ACF6186178207863
:103AA000023406F083FCA642F8D1314B314A196842
:103AB00003201140A022D2020A431A608022196812
:103AC00092040A431A6019682B4A1140802292031B
:103AD0000A431A60294B2A4A934200D8012007F072
:103AE0005FFE07F0C5FE08F05BF8287808F078F96B
:103AF000039B1878C0B208F083F807F059FE2149FB
:103B0000042008F00DF906F06BFE00F0B1F800F0AB
:103B1000FBFD00F08DFE00F01BFA002011B0F0BD9F
:103B200000932100174A042007F0D2FE8023DB0512
:103B30009C62FFF78BFC5DE74A0AFF1F34F00040F0
:103B40002447FF1FC064FF1F480AFF1F490AFF1FC9
:103B5000680AFF1FBCF0004000E100E0FF00FFFF2B
:103B60002847FF1FAC59FF1F2857FF1F50BE0011E9
:103B700014F00040FF7FF8FFFFFF9FFF6072FF1F00
:103B80000080FF1F3B00010870B5002529492A4A23
:103B90002A484D6308CA1B051B0DED188242F9D156
:103BA0000022274B8B63274B08211A628022264B69
:103BB0009205DA67254BDA688A43DA60244A12787C
:103BC000012A03D09A6823490A409A6002202249B8
:103BD000EE240A68E40082430A600121DA686C433B
:103BE0008A43DA600F3008F0C3F8112007F0C0FEF6
:103BF000112007F0EDFD194A200C040064239042C7
:103C00000AD8FA220023D200904205D9144B0A2187
:103C1000C01808F015F9C3B2124A1372124BD480BF
:103C20001B78002B04D1114B1021187807F038FFB6
:103C300070BDC046000005400806054080060540EE
:103C4000FF01000000F0004004E100E03CF0004013
:103C50004A0AFF1FFFDFFFFF00380040B70B0000DC
:103C600030F8FFFFA864FF1FE466FF1FE064FF1F3A
:103C7000002210B51100112007F03AFE10BD00001F
:103C8000F8B5002301250826394F3A4C3B62E3681A
:103C90001120AB43E360E368B343E36007F068FEE1
:103CA000112008F065F8112007F0E2FF4023226898
:103CB00029001343236080236268DB02134363609F
:103CC0008023A26830001343A360A3682A4A1340EC
:103CD000A3608023A2689B0113431022A360236C7E
:103CE00093432364236C2B43236480231B013B6297
:103CF000226B224B10271A402263626B1A406263C8
:103D0000A26B1A40A263E26B1340E3631C4AE368B0
:103D10001340E36006F030FC2900300006F05AFC46
:103D20008023184A5B00516C11200B43536407F049
:103D3000BFFEFD21C720144B144A89005A50A36BC3
:103D400080003B43A363E368114A1E43E660E368D7
:103D50001D43104BE56019581140802212020A439E
:103D60001A50802292051A600B4B5F63F8BDC04663
:103D700000F000403CF00040FFFFDFFFEFFFEFFFEF
:103D8000FFFF7FFF003800400000FF1F893B00114C
:103D9000FF00FFFF00E100E00000054030B503A890
:103DA00004880B20002C0ED14968074D087849780B
:103DB000090201430A20A94205D1012120001980EE
:103DC000024B1B7A137030BD192A0000A864FF1F34
:103DD000F7B5150008AA16884A680F4F147852786C
:103DE000120222430A24BA4214D10122DBB2019208
:103DF00000962A0007F044FC041E0BD1074B1B68F9
:103E0000002B07D068782A780002104342425041C4
:103E1000013098472000FEBD022900002C64FF1FDE
:103E200030B5012503790400BFB02B4212D00A49F6
:103E3000408806F091FF28420CD06A46074B69463D
:103E40005B8D55801380064B60881B7A13710022AE
:103E500004F074F83FB030BD2464FF1F5843FF1FC7
:103E6000A864FF1F10B50549054806F02BFF042183
:103E7000044A054806F0E8FE10BDC0462464FF1F52
:103E8000FFFF000080BE00115843FF1F10B502481D
:103E900004F0D6FE10BDC046213E0011062310B529
:103EA000837010330371443B43712A33837144336D
:103EB000C37100230222012103720E4B0270417074
:103EC0001C8881724472197A0273C1729A784273A3
:103ED000DA7882730322C2731A7902745A794274AF
:103EE0000C2282749A79C274DB7903751123C37032
:103EF000152010BDA864FF1F10B5142007F088FE20
:103F0000124B14220021186007F0F2FD002007F088
:103F100017FD012007F044FD022007F081FD03207A
:103F200004F032F9042006F047F9052003F070FB95
:103F3000062004F03DF8072001F038FA082006F0CA
:103F400063FE092001F020F810BDC0463064FF1F59
:103F500010B507F0D5FC012007F04AFC07F090FEF1
:103F6000002010BD094B10B50400984205D001296E
:103F700004D12000064906F0A5FE10BD0229FCD19F
:103F8000013904F01BFE0028F3D0F6E7FEFF000025
:103F90005664FF1F70B50D7A100004AA2C00168815
:103FA00010221440154220D1002E20D10A78022A76
:103FB00018D14A68517815780E4A0902294391426E
:103FC00005D00D4A914209D01C800A2404E0142235
:103FD0000A491A8007F0A4FC200070BD0C22084991
:103FE0001A80F7E71C800124F6E70824F4E70B2485
:103FF000F2E7C046F3FF0000F4FF0000A845FF1FF2
:104000005CBF001110B504000749084806F05AFECD
:10401000074804F055FD0020E40704D50721054AB0
:10402000054806F011FE10BD5664FF1FFFFF00009B
:10403000653F0011C4BE00119C43FF1F00B50C4B2F
:10404000BFB01A780B4901A800F0ACFC6B4680B2F7
:104050005880002809D06A46074B69461B881380A0
:10406000064B0022188803F069FF3FB000BDC04630
:104070003464FF1F3564FF1FF643FF1FFE44FF1F1C
:1040800000B50C4BBFB01A780B4901A801F09CFE9B
:104090006B4680B25880002809D06A46074B6946B3
:1040A0005B8D1380064B0022188803F047FF3FB05A
:1040B00000BDC0465E64FF1F5F64FF1F9C43FF1F7F
:1040C000FE44FF1FF7B50E00377A1C0008AB110045
:1040D0003D001A8820231D401F423CD13378022B1B
:1040E0003BD173681F785B781B023B431E4FBB427A
:1040F00008D01E4FBB4214D01D4DAB4221D00A2523
:104100002800FEBD002A2AD1142C2AD82200F068EB
:1041100007F006FC174B1C70012CF1D9FFF7B0FF1C
:10412000EEE7002A1BD1202C1BD82200F06807F0F4
:10413000F7FB114B04211C70104B187807F0B0FCF2
:10414000DEE7E3B20124009201940A00310007F097
:1041500097FA0500D4E70825D2E70125D0E70B251B
:10416000CEE70D25CCE7C046F3FF0000F4FF0000CA
:10417000022900005E64FF1F3464FF1FE064FF1F1C
:10418000332310B5040003700A220749013007F0F9
:10419000C7FB064B0F201B681A0AE37222731A0C26
:1041A0001B0E6273A37310BDA864FF1FD064FF1FB2
:1041B00030B5012503790400BFB02B4213D00B4961
:1041C000408806F0C9FD28420DD06A46084B01A878
:1041D0001B881380FFF7D4FF6B4658800022694686
:1041E000608803F0ABFE3FB030BDC0465664FF1F91
:1041F000F643FF1F10B5024804F022FD10BDC04673
:10420000B141001170B5160004AA148805AA1578EA
:104210004A685078117800022A4A08438018052815
:104220004BD807F0DDFC03131E29343F0720032C75
:104230000BD80422121BAA4200D92A0022491A8054
:104240003000091907F06CFB002070BD0720112C0D
:10425000FBD81222121BAA4200D92A001B491A803D
:10426000EEE707200E2CF0D80F22121BAA4200D92D
:104270002A0017491A80E3E70720032CE5D8042217
:10428000121BAA4200D92A0012491A80D8E7072037
:10429000032CDAD80422121BAA4200D92A000E49A4
:1042A0001A80CDE70720032CCFD80422121BAA4284
:1042B00000D92A0009491A80C2E700220A201A8080
:1042C000C3E7C046DCD5FFFF0FBF00117C64FF1FB2
:1042D000FFBE0011FABE0011F5BE0011F0BE0011C4
:1042E00010B50D21024A034806F0AEFC10BDC046D1
:1042F000E4BE00110C44FF1FF0B50024274E85B02A
:104300003000B47100F0E2F8254D264BEA89297C93
:104310009A422FD10423300003AA00F057F9040079
:10432000300000F011F90123B371002C34D16B4639
:1043300099892B68C9BA4B4329891B4A1B145B18FE
:1043400053806B46D9896B6849BA89B24B436989F6
:104350001B0C5B181548191C1BB2834200DD011CA5
:104360000B0400D5002113889180013313802000B5
:1043700005B0F0BD0227220003AB3000009700F02B
:10438000F7F80E230400297C0122300000976B44CB
:1043900000F0EEF80443C3E71C00E8E7E444FF1F25
:1043A0009064FF1F83050000A864FF1F0F27000013
:1043B00073B5234E300000F089F8224D07236A467A
:1043C0003000297C00F002F904003000002C33D1C9
:1043D0006B461B787F2B2FD800F0B6F86B46D87849
:1043E000F02302041B031A406B469B8816495BBAF4
:1043F0009BB21A432B68000953432A891B0C9B1854
:104400004B806B465A789B7812031B011A436B68EA
:10441000024353436A891B0C9B180C481A1C1BB29D
:10442000834200DD021C130400D500220B888A8021
:1044300001330B80200076BD00F086F80124F9E7F7
:10444000E444FF1F9064FF1FA864FF1F0F270000B4
:1044500070B5114C237C002B0FD0382B0ED10F4D93
:10446000280000F033F8CC23AC222800217C9B01EB
:1044700000F0F4F8280000F067F870BD084BE289FE
:104480009A42FAD1054D280000F020F800222800B9
:10449000217C00F0C5F8EDE79064FF1FE444FF1FA6
:1044A0008305000010B5084B1A7C002A09D05B690F
:1044B000002B06D09847041E01D0FEF7A1FD200076
:1044C00010BD0124F9E7C0469064FF1F70B5C179A3
:1044D00005000C00631E9C411A4BE402E4184900DD
:1044E0000460C9B2007906F0ABF8E979687949004F
:1044F0000131C9B206F0A4F8E8790930C0B207F07A
:10450000B7FB0023E36661332360AA795B3B002A93
:104510000ED022689A43023B134323600A23E361CF
:104520000733236200232363A3630133E36370BD76
:1045300022689A43022313432360462363610633B0
:10454000A361EFE70050004070B500250400036848
:10455000DD66C0790930C0B207F00AFA2900207977
:1045600006F00AF82900607906F006F870BD000030
:10457000F8B51E0006AB1D78002304681700E3663B
:10458000616007F005FC01238022E3662B002761B0
:104590005200013B08D207F0E3FA08200A4A1168EA
:1045A000002D03D12800F8BD2261F2E7236F0342FA
:1045B00003D02369013D3370013613685B1A032B66
:1045C000EED90125EEE7C0466008FF1F70B51C005C
:1045D000002305681600EB66696007F0D9FB01232C
:1045E0008022EB6623005200013B08D207F0B8FAA4
:1045F00008200A4A1168002C03D1200070BD2A61EE
:10460000F2E72B6F034203D02B69013C3370013674
:1046100013685B1A032BEED90124EEE76008FF1F35
:10462000002370B504681500E366616007F0B0FB15
:104630000123E366256107F093FA8020064A800093
:104640001168636B034205D113685B1A032BF8D919
:10465000012070BD0020FCE76008FF1F70B51D0041
:10466000002304681600E366616007F091FB0123F4
:10467000E36626610F33626B1A42FCD02B0A23617A
:104680001023626B1A42FCD0EDB2256107F068FA84
:104690008020074A80001168636B034205D11368CC
:1046A0005B1A032BF8D9012070BD0020FCE7C0463F
:1046B0006008FF1F70B51E00002305681400EB663C
:1046C000696007F065FB0123A619EB660F33B4425E
:1046D0000ED107F045FA80200A4A800011686B6B02
:1046E00003420CD113685B1A032BF8D9012070BD6B
:1046F00021782961696B1942FCD00134E7E7002079
:10470000F5E7C0466008FF1F10B5084CE368002BB2
:1047100008D1074B1B685B045B0C0A336360054BD5
:104720001B68236007F08CF9A06010BDD064FF1FE8
:10473000C8F00040CCF0004010B507F029FB0F4B4B
:10474000996A9A6A8A42FBD10D4C6268A0688A18FD
:10475000121A531E884200D31300A1602168DA0B9D
:1047600052185B0407495B0C636022600B60064BC8
:104770001A6007F0F5F9206810BDC04600F000404F
:10478000D064FF1FC8F00040CCF0004070B51F4C53
:1047900023793F2B01D93F2323711D4B22791A70B6
:1047A0001878C0B207F024FB18231A491A4A0B8064
:1047B0001A4913800B805380A379194980200B80FC
:1047C0000C21938001334B430001191C834200D913
:1047D000011C144BD18019806379002B11D1013356
:1047E0006371237A012B01D8022323726279237A21
:1047F0000D4853430A21584307F022FB0B4D286014
:1048000070BDA02BEDD9A023EAE7C046C464FF1F0A
:10481000480AFF1FFC44FF1FD046FF1FFA44FF1F3A
:10482000B066FF1FF844FF1F71020000B464FF1F51
:10483000F8B513210020FEF7D1FD114C011E114DDA
:1048400009D10C22104BC1CBC1C4280007F050F98C
:10485000FFF79CFFF8BD0C2220000C49FEF792FDEB
:104860000C2802D0084B43CB43C40C222800084933
:10487000FEF788FD0C28EBD00C220021E5E7C046AE
:10488000C464FF1F9064FF1F50BF0011FC0C0000A8
:10489000F50C0000F0B51D4C8022A54404008820D2
:1048A00069465201400507F003F8902212016A445C
:1048B0001300200032C832C316C816C38023144C1C
:1048C000144FA6689B033343A3603B6007F0B0F826
:1048D0008823A0685B05C01807F0A2F9002588238B
:1048E00029008022A0685B05C01840196944520065
:1048F00007F0EEF980230135FF355B019D42EED1D3
:10490000A6603E60044B9D44F0BDC046FCEFFFFF37
:104910004046FF1F9808FF1F04100000F0B5040078
:1049200087B0002825D0684607F012F81B4C0228F3
:1049300006D106226946200007F032FA002816D078
:104940006946002301250F262F00E25C0133100980
:104950001030874038002F00324097403A00024321
:104960004A610439062BEFD16846FFF793FF07B081
:10497000F0BD182269460A4806F09AFF6A46A3006D
:10498000D358013305D01822FF21684607F0B0F84C
:10499000EAE70134062CF1D1E9E7C0466509FF1FBB
:1049A00000090011F0B5002504000E0085B0AA42F0
:1049B00000D186E04B1C087801934B7889783779D1
:1049C00009021943F3783F061B040B431F43039767
:1049D00020706570252800D196E033D8112813D8AF
:1049E00006F0BEFF69002501250125012501AA0069
:1049F000B800B1002501250125012501250125016A
:104A000025012501FF001F01232800D1D8E0DB2864
:104A100000D02EE1042A00D8ACE01025052A05D0EC
:104A2000551F2A003800711D06F07AFF052231005B
:104A3000200006F075FF2A003900601D06F070FFA7
:104A400005353EE0562859D010D8332800D19DE0D6
:104A5000552839D02628DAD19C4B2900132218007A
:104A60001D0007F045F8FEF7CBFA5CE0712800D195
:104A700077E0722800D180E0602800D18BE0DC284C
:104A8000C5D1022A00D875E07378BFB26370B378DD
:104A9000A370032A05D0033A390092B2F01CFEF746
:104AA000ABFB10223900E01CFEF76CFCC51C002893
:104AB00007DA60705CE00C222000854906F030FFC8
:104AC0000C25280005B0F0BD013A824D0C2A13D800
:104AD000002A0AD02800019906F022FFFFF756FEAF
:104AE0000C2228007C49FEF787FB29000C22601C61
:104AF00006F016FF0D25E4E70C22EBE7754D774B2A
:104B00002A0043CB43C2E9E7013A704D0C2A11D881
:104B1000002A08D00199280006F002FF0C22280084
:104B20006F49FEF769FB29001322601C06F0F8FEAE
:104B30001425C6E70C22EDE705226A49601C06F041
:104B4000EFFE0625BDE712226749601C06F0E8FE6D
:104B50001325B6E708226549601C06F0E1FE092529
:104B6000AFE77178F72905D8614B188801F088FD07
:104B70000225A6E7FF236370FAE75E4B012A03D004
:104B800072785A706270F3E75B78F4E72000FFF701
:104B9000F7FA050095E7013A574D072A0ED8002A83
:104BA00005D00199280006F0BBFE01F047F8290066
:104BB0000722601C06F0B4FE082582E70722F0E712
:104BC000042A04D94D4D2F6006F03AFFA860FFF784
:104BD000B3FD0422039003A9601C06F0A1FE052585
:104BE0006FE7474D062A15D906222800019907F0DC
:104BF000D7F800280ED006220199280006F090FE72
:104C0000062240492800FEF7F7FA0123394A517875
:104C10000B43537029000622601C06F081FE072515
:104C20004FE7012AA6D07078FFF778FEA0E70128A9
:104C300000D0ECE6931E344F1A2B04D87378002B67
:104C400009D100F015F9314B39001D78601C6A1E3E
:104C500006F066FE35E7551E2A000199380006F079
:104C60005FFE2B49AAB23800FEF7C6FA00F036F90B
:104C7000E9E7DA281DD1042A00D87BE7082A15D9EC
:104C8000B37972791B021343F27912041A43337A0F
:104C90001B0613433B603B68052231002000039351
:104CA00006F03EFE0422601D03A956E7FE23637052
:104CB000F1E7DE2800D05DE7511E012A01D1002571
:104CC000FFE6019800F0A0FFF9E7C0469064FF1FDF
:104CD0005CBF0011C464FF1FFC0C000050BF00113A
:104CE000F50C00009C64FF1F7C64FF1F4446FF1FFF
:104CF000FE44FF1FC064FF1F9945FF1FD064FF1FC4
:104D00006509FF1FADAC0000C366FF1FC166FF1F32
:104D1000AEDE000070477047020010B5094B0A3242
:104D2000094C92B2DA815A8298811882207802F076
:104D30000DFB0422054B012120781A7006F0B0FE0D
:104D400010BDC046CE45FF1F0E67FF1F0D67FF1F3A
:104D5000013870B5042809D806F042FF0309280875
:104D60001200234B0221187806F09AFE70BD204BEA
:104D70000821187806F034FE00221E4B1A72F5E75F
:104D8000802200241B4B1A4D52001A8108211A68F8
:104D90002878DC7206F074FE2100287806F0B8FF4F
:104DA000012000F051FE00F049FFDFE7104B082121
:104DB000187806F015FE1048FFF770F80F4B104AF0
:104DC0009B79002093800F4A13808022094B520068
:104DD000D8721A8100F038FE00F030FF0A4B5B7881
:104DE000002BC3D0094A136007F022F8BEE7C04683
:104DF000E064FF1FB464FF1F0745FF1FC464FF1F6B
:104E0000D046FF1FB066FF1FC064FF1F34F0004094
:104E100010B501290BD1012809D1054B1B78002BB6
:104E200005D02622034B04485A72FFF775FF10BDC8
:104E3000E466FF1FB464FF1FC40900000300F0B55F
:104E40000A4D8E18B14202D152008018F0BD0C7884
:104E50002F6824093C5D0F271C700C7801313C4001
:104E60002F683C5D5C700233ECE7C046F444FF1FE2
:104E70000D22114B10B51A700C23104C10492370E1
:104E8000093A033B0F48637006F04AFD2D230122C7
:104E90000D490E48A371FFF7D1FF01220C49FFF71E
:104EA000CDFF01220B49FFF7C9FF00220A4910007C
:104EB000FEF7A2F910BDC046E066FF1FC166FF1FE6
:104EC0000FBF0011C366FF1F6709FF1FC866FF1FE2
:104ED0006609FF1F6509FF1FAEDE000070B5124CAA
:104EE000132220001149FEF74DFA114D002817DD5D
:104EF000AB78002B14D0431C2B7009236B7000235C
:104F000000190370287829000130C0B206F0E0FDD6
:104F1000297822000139C9B2002005F0B3FD70BD27
:104F2000FFF7A6FFEEE7C046C366FF1FAEDE000038
:104F3000C166FF1F10B5114B1A781870002A0ED0E9
:104F400000280BD10E4B1A78062A07D85423D340D9
:104F5000DB0703D50B4B187802F0F8F910BD0028D9
:104F6000FCD0074B1B78012B02D0033B022BF5D85A
:104F7000044B0121187806F093FDEFE7E466FF1F6C
:104F80000D67FF1F0E67FF1F70B54A4E4A4A4B4917
:104F90003070012005F002FC00F0B4FEFEF730F89E
:104FA00006F026FD032246494648FFF747FF2D2419
:104FB000030004221C7044490130FFF73FFF3023F7
:104FC0000470424D424C437083702E3B06222000F9
:104FD0004049EB87FEF7D6F9062813D0200006F0EB
:104FE000B7FC022809D00321200006F0E9FC8D233C
:104FF000E3706E3B2371193363710622200035493B
:10500000FEF7FAF8344B1B68FC335C64FFF766FF6D
:105010000020FFF78FFF314C314A0121314B1278CC
:10502000207802F055F9304A304B12780021207870
:1050300002F04EF901222E4B1A702E4B9B78552B05
:1050400031D12D4B3B325A722C4B2D4AAB81EA8128
:105050002B826A822021307806F002FD0120404236
:1050600005F05CFD0120404205F0F8FDFFF738F93E
:10507000FEF7F8FE00F0A6FC01204042FEF7C2FF5A
:10508000012006F005FCF72001F0DEFA012130785E
:1050900006F006FD307802F0B5FA1A4806F0F0FB8B
:1050A000FEF7EEFD70BD6422174B5B7953431A0087
:1050B0000A32CBE7E064FF1F154D0011114E0011BD
:1050C0004446FF1F7C64FF1F9C64FF1FCE45FF1FEB
:1050D0006509FF1FADAC00006C67FF1F0E67FF1F67
:1050E0002645FF1F0745FF1FE066FF1FC166FF1F24
:1050F000B266FF1FC064FF1FB464FF1FC409000035
:10510000CE090000E264FF1FC464FF1FF8B50A0067
:1051100020230D001A40194257D0574B1B78002B03
:1051200050D0FFF709FB554B554C564E99686268B5
:10513000737A8A1ADB039A4202D36160FEF7A0FDFC
:10514000327A217A531EDBB2994205D1FFF780F9FA
:10515000002000F0A9FD0FE09142F9D30023237253
:10516000FFF7A0F9012000F09FFD474F3800FEF740
:1051700095FE390006F044FB637A002B1FD0013BFB
:10518000DBB26372002B1AD1404B9B78552B01D1B7
:1051900006F04EFEE37A002B0CD000233C4A3A4F37
:1051A000E3721388380001331380FEF777FE39006D
:1051B00006F026FB642370795843FFF7ADFD237A90
:1051C0000133237220206840F8BD0BB2002B0ADAAD
:1051D000304B187806F0ECFD002801D006F0D0FC2A
:1051E00080200002EFE70224214206D0244B012058
:1051F0001A72FFF79FFE2000E5E70B071ED5FFF7A9
:105200009BFA1E4B1E491F4C98684A68637A821AA3
:10521000DB039A4202D34860FEF732FDFFF742F902
:10522000FFF716F9012000F03FFD00F0E5FB2368D1
:10523000DB0701D5FEF7DEFF0820C4E7102421427A
:1052400006D00D4B1B78002BD5D1FEF71FFED2E701
:105250000124214207D0104800F06CF806F060FCF1
:1052600000F008FDC7E70424080020402142ABD02D
:10527000FEF7E4FEBFE7C046E466FF1FD064FF1FF1
:10528000B464FF1FC464FF1F0745FF1FC064FF1FF6
:10529000A864FF1FE064FF1FEC44FF1FF0B51B4B29
:1052A0001B4F1B883A8804001A4E1B4D85B09A424A
:1052B0000DD832889A420AD3184B1A882B889A4202
:1052C00005D1174A174B12881B889A421BD005201C
:1052D00001F010FA3B8802AA1380338801905380B2
:1052E0002B88114D93800F4B02A91B88D3800F4B45
:1052F0002A78188802F02CFF0D4B08212878019A93
:105300001C7006F07DFB05B0F0BDC046AE66FF1F09
:10531000FC44FF1FFA44FF1FB066FF1FAC66FF1F6F
:10532000AA66FF1FF844FF1F0E67FF1FFE44FF1F02
:10533000A866FF1F13B50C4B1C78002C11D1002858
:1053400001D00A4B18600A4A0A4B11780A4A1078B1
:105350000A4A01920A4A0092002205F08BFA2000C4
:1053600016BD1124FBE7C0460D67FF1FA466FF1F93
:105370000C67FF1FFC66FF1F0E67FF1FE866FF1F1D
:10538000EC66FF1F10B5064B12201B78052B06D1CB
:10539000044B13221988044B187801F087FB10BDC9
:1053A0000D67FF1FFE44FF1F0E67FF1F10B500248F
:1053B0000122114B52421870104B1C70104B1A8076
:1053C00002F020F904220F4B21001A700E480C3213
:1053D00006F0DEFA102221000C4806F0D9FA072266
:1053E0000B4B1C600B4B1C700B4B1C700B4B1A7047
:1053F0000B4B1C7010BDC0460E67FF1F0D67FF1FD3
:10540000FE44FF1F0C67FF1FFC66FF1FEC66FF1FBB
:10541000E866FF1FC066FF1FBF66FF1F0045FF1F36
:10542000BE66FF1FF8B5174C0600257806A81424A1
:105430000078052D23D1B41F134FA5B21824BD4207
:105440001DD88D1FADB2BD4219D8FA256D00AA42F4
:1054500015D21D000D4F0A3DADB2BD420FD80C4C08
:1054600026800C4C21800C4900240A800B4A1380B2
:10547000FFF714FF0A4B0421187806F0B1FA200058
:10548000F8BDC0460D67FF1F790C0000750C0000C9
:10549000FC44FF1FFA44FF1FB066FF1FF844FF1FC4
:1054A0000E67FF1FF0B50BB20D0089B0002B00DBBB
:1054B00070E1A44E307806F07BFC041E50D00378D7
:1054C000A22B00D122E1D02B1AD0912B45D14378C9
:1054D0000E2B42D19C4B82889A423ED19B4A8368D4
:1054E0001278052A39D1032018567F2835D0984BD9
:1054F0001B68002B31D05B68002B2ED098472CE026
:105500008078072829D806F06BFB0428183F3F74E1
:10551000A8D86378002B0CD101218C4B19708D4BCE
:105520001A78002A5BD08C4B307801F0D1FE00282D
:1055300055D00722854B1A7051E061780029F8D1C7
:10554000E378002B11D0854A854B1278307801F032
:10555000BFFE60706378002BEBD1200006F010FBDB
:1055600080200002684009B0F0BD784B1B78022B08
:10557000F3D00121307806F0DBFA0028EAD10121CE
:10558000307806F08DFAE5E76378002BD1D16F4FC4
:10559000032807D13B78052B02D101333B701EE075
:1055A0000223FBE76F4B1A886F4B0293002A0BD044
:1055B0001B78002B03D00121307806F021FA3B78CC
:1055C000062B04D1013BE9E7029B1A70F7E7042B95
:1055D00041D10121029B3078197006F061FA5C4BD1
:1055E0001B68002BB9D01B68002BB6D0574A107827
:1055F00084E76378554F002B27D10622211D5B4895
:1056000006F08EF962895A4B5A491A80A2895A4B80
:105610001A80E3890B800521397058490A80584A5D
:105620001380228A574B1A80574B1B78012B09D1C4
:105630001F2001F05FF8FA229200424304213078E3
:1056400006F0DEF90022484B75E7312B00D070E7F9
:105650000022454B1A700323A0E70622002143488D
:1056600006F096F90023454A04211380444A307815
:105670001380444A138006F0B3F90821307806F00D
:10568000AFF9A379083B5A425341304A03331370B0
:10569000304B1B78002B06D0334B30781A78002A19
:1056A00006D001F053FE0122314B52421A8096E798
:1056B0000121197006F0F4F9F5E70821307806F0B9
:1056C0008FF96378002B00D047E72C4B2D4F0293C6
:1056D000E388029A04211380294B307803932389AD
:1056E000039A138063893B8006F022FA002800D0D9
:1056F00033E7264B1B68002B00D12EE70399029855
:105700003A88098800881B68984726E74379132B55
:1057100000D022E70389012B0AD11D4B1B78022BF5
:1057200006D10821307806F05BF9FFF72BFE14E76D
:10573000052000F0DFFF08210200307806F060F954
:105740000BE7C0460E67FF1F051400000D67FF1F23
:10575000A466FF1F2645FF1F0745FF1FE066FF1FCA
:10576000C166FF1FE266FF1FE466FF1FB366FF1FEF
:10577000FE44FF1FBA66FF1FBC66FF1FAE66FF1F19
:10578000AC66FF1FAA66FF1FB266FF1FA066FF1F61
:10579000A866FF1F8020C001014200D0E2E6CB07CF
:1057A00031D5324B1B78002B1DD0314E05AC3378F0
:1057B000052B1AD1023B23702E4B21001B7823723C
:1057C0002D4B1B7863722D4B187801F025FD0028B6
:1057D00009D007202A4B30701B68002B03D01B68B0
:1057E000002B00D098470120BCE60E20254B062256
:1057F0001B7825492370254B1B78637002ABC018BA
:1058000006F08EF8D8E7022308001840194209D0A4
:10581000174B1B78052B03D11D4B188805F0D0FFC3
:1058200002209FE60424214203D0FFF737FD200029
:1058300098E6082308001840194200D193E6154B5A
:105840001C78012C03D0022C0DD008208AE6124BC4
:10585000124A134913481B8812880988008800944B
:10586000FFF7E0FDF1E7FFF78DFDEEE7E466FF1FD0
:105870000D67FF1F0045FF1FBE66FF1F0E67FF1F5E
:10588000A466FF1FC066FF1F0145FF1FBF66FF1F05
:10589000FE44FF1FA866FF1FF844FF1FB066FF1FEE
:1058A000FA44FF1FFC44FF1F10B502A804880B2018
:1058B000002C10D1496808784978090201430C4846
:1058C000814209D1022119800A4B59881170DB7875
:1058D00000205BB2537010BD074C0A20A142FAD1E0
:1058E00002211980034B998811705B79F0E7C0465B
:1058F0006E2A0000A864FF1F6F2A0000F7B515008C
:1059000008AA16884A680F4F147852781202224368
:105910000A24BA4214D10122DBB2019200962A0075
:1059200005F0AEFE041E0BD1074B1B68002B07D001
:1059300068782A780002104342425041013098476B
:105940002000FEBD022900002067FF1F30B50125A1
:1059500003790400BFB02B4227D01549408805F0D9
:10596000FBF928420DD06A46124B69465B8D1380C5
:1059700002235380104B5B8893806088002202F0E2
:10598000DDFA0E49608805F0E7F9C0070DD56A46D3
:105990000B4B69461B88138002235380064B9B8860
:1059A00093806088002202F0C9FA3FB030BDC04643
:1059B0001867FF1F2845FF1FA864FF1F1067FF1F00
:1059C0008245FF1F10B5074C0749200005F07AF902
:1059D0002000064905F076F90721054A054805F03B
:1059E00033F910BDFFFF00001867FF1F1067FF1F8E
:1059F000DCBF00112845FF1F10B5024803F020F955
:105A000010BDC0464D5900110221430888400B408B
:105A10000A31084003430E20024AD17881430B43E8
:105A2000D37070479945FF1F064A1379410705D582
:105A300080210B4380011371907170477F210B40CF
:105A4000F8E7C0469945FF1F054A5378002803D060
:105A500080210B43537070477F210B40FAE7C0460B
:105A60009945FF1F0F21114BDA780A40DA70502850
:105A700010D901310A43DA702022D9780A43DA704A
:105A80004022D9780A43DA708022D97852420A43F8
:105A9000DA7005E03C28EFD82828F1D81428F3D88C
:105AA0000122D9780A43DA707047C0469945FF1F32
:105AB000F8B57F23324D04006E789E43314B9842F7
:105AC00005DD76232B70363B33436B70F8BD2E4BD0
:105AD000984203DA58232B701433F5E783B21A0087
:105AE00000215F32294892B2294F297082422DD974
:105AF000A9708C4203DA5B421CB220232B70053460
:105B000020B20A2106F09CF904B2FA239B009C42C1
:105B100033DB80232A785B4213432B7064212000FF
:105B200006F08EF90A2100B205F072FE09B22A7859
:105B30007B5C13432B700A21200006F081F90A21B7
:105B400000B205F065FE09B27B5C0AE08022AA7013
:105B5000002CDADA5B421CB220232B705F23092C65
:105B6000E9DC1E430A2120006E7005F051FE09B2E7
:105B7000AA787B5C1343AB70A8E7632CCEDCEDE71F
:105B80009945FF1F1B4E00001DFCFFFF2A08000067
:105B900006C000117F23F7B5194FCD013E790400EF
:105BA0009E433E71EDB2632806DD093B33433B71F2
:105BB00040231D437D71F7BD0300093304DA5823E8
:105BC00033433B716C23F4E70E4B019300280BDA4F
:105BD0000423444224B23B710A21200005F018FE40
:105BE000019B09B25B5CE4E70928F5DD0A2106F0B8
:105BF00027F9019B00B21B5C1E433E71ECE7C046D7
:105C00009945FF1F06C00011F8B50A4F05003B7803
:105C10000E00002B0CD0084C2000FEF757FC330080
:105C20002A0020003978FEF745FD2000FEF78CFCA5
:105C3000F8BDC0462C67FF1FA045FF1F70B50A4E78
:105C40000A4D07223100280006F0AAF8002809D0E2
:105C5000074C31000722280005F062FE08212000D1
:105C6000FFF7D2FF70BDC0469945FF1F2567FF1F94
:105C70002467FF1F7F2210B50A4B59789143033ADE
:105C80001A70103A0A435A7078220E219A70DA7804
:105C90008A43DA7006221A7129325A71FFF7CEFF51
:105CA00010BDC0469945FF1F10B5002824D0134CE5
:105CB0000A210223E05E06F0C3F800B2FFF7F8FE07
:105CC0000423E05E642106F0BBF8012100B2FFF777
:105CD00061FF207AFFF7C6FE0320FFF795FE002044
:105CE000FFF7A2FE064B1878053843425841C0B270
:105CF000FFF7AAFEFFF7A2FF10BDC046A864FF1F72
:105D00000D67FF1F70B50024094D2800AC71FEF728
:105D1000DDFB10233E212800064AFEF7CBFCA04203
:105D200000D13E34044B28001C70FEF70DFC70BD02
:105D3000A045FF1FF6BF00112C67FF1F0200F0B542
:105D400001270A480A4E51188B1A002B00DCF0BDBF
:105D5000082415784308684038404000805B013CC7
:105D600058406D08002CF5D10132EDE7FFFF00002F
:105D700016C00011F0B500250F269D4200DBF0BDD6
:105D80004C5D070944403440A400A05801357840D8
:105D9000F3E70000F0B589B06A460D000B000F274D
:105DA000110010351C780133260024093E4016707E
:105DB00054700232AB42F5D12023024AFFF7DAFFDA
:105DC00009B0F0BD1CC00011F0B54E780B7889B059
:105DD00036020C00170001901E43012A61D9954B31
:105DE0009E4200D877E001339E421CD1062A17D18B
:105DF000CA788B7812021A430B791B0413434A7931
:105E000012061A438C4B5A6100221A705A808B4A30
:105E10005A608B4A9A608B4ADA60002009B0F0BD64
:105E200088225205EEE7884B9E423CD182498B780E
:105E3000002B00D0F6E00C2A31D10F22A378934337
:105E4000E278120213432279120413436279120694
:105E500013434B60E279A07912020243207A0004D6
:105E60001043627A12060243CA60E27AA07A1202F2
:105E7000024376484A81834208D804236E4914229B
:105E800001980B7005F04CFD1420C7E71201D218E1
:105E900089235B059A42F0D801238B70BDE7022A63
:105EA000FAD00523EAE76A4A01239642E6D1FFF7D2
:105EB00069FA052F0CD9E378A2781B0213432279E3
:105EC00012041A4363791B061343624A0393136057
:105ED00005F0AEFFA1E7584D2B78002B9DD1AB7894
:105EE000002B00D1A0E02B8901339BB20093B34279
:105EF00000D091E0132AD4D9CF7C8B7C3F021221B1
:105F000020001F43FFF71AFF874200D08EE0002ECB
:105F10003DD1E378A2781B0213432279E968120489
:105F20001A4363791B06134303930A228B4212D14F
:105F3000FF23A370E370237163716B89002B09D178
:105F4000E37B227C1B0212041343A27B13431B0935
:105F500001336B8100226B89002B8ED0002A67D120
:105F6000686837013818000B6B690003039098428A
:105F700005D9686105F054FEEB780133EB70686871
:105F80001022A11C381805F0A3FE2E8145E76F8969
:105F9000009A7B1E9BB293423AD1E278A378120218
:105FA0001A43237905A81B04134362796C6812060F
:105FB0001A43EB6800920392211D0C22049305F012
:105FC000AFFC0120260004A940421036FFF7E2FE94
:105FD000013F012F17D1009A0B232861824200D084
:105FE0004CE704221C49200005F072FE042203A99C
:105FF000686805F05DFCE968039AFF23914200D1CF
:106000003CE7F73B3AE73100FFF7C4FE1036DFE725
:106010000923B742A4D831E7009BB34200D9FCE67C
:1060200007232BE7022329E7032327E7062325E796
:106030000A2323E7FFFE0000A845FF1F000001110F
:10604000FFFF00005048593601FF0000FFFF00111C
:1060500002FF000034F00040B445FF1F10B5034CB0
:106060000B000122210000F06BFA10BD1D6200112F
:106070000B8870B506000D000224162B11D92B00D9
:106080000322094900F05CFA041E0AD1074B2A8852
:106090001B88191C934200D9111C300089B200F0F2
:1060A000EFFA200070BDC046496200118667FF1FED
:1060B00010B54A780400013A0B000220012A07D8E3
:1060C0000A78002A04D005222000024900F038FA9C
:1060D00010BDC046776200110A7810B50B000400AD
:1060E0000220002A04D007222000024900F028FAEA
:1060F00010BDC046236300110A7810B50B000400E0
:106100000220002A04D009222000024900F018FAD7
:1061100010BDC0468963001110B5034C0B000B2263
:10612000210000F00DFA10BDB963001110B5034C49
:106130000B000D22210000F003FA10BD2B640011AA
:1061400010B5034C0B000F22210000F0F9F910BD2F
:10615000856400110A7810B50B0004000220002AA3
:1061600004D011222000024900F0EAF910BDC04617
:1061700095640011002310B51322190000F0E0F916
:1061800010BD000010B5034C0B001722210000F0D9
:10619000D7F910BDE7640011002310B519221900CA
:1061A00000F0CEF910BD000010B5034C0B001B220F
:1061B000210000F0C5F910BD21650011F7B58489F3
:1061C0000D0006000121002C22D000238268D35646
:1061D0001778002B1EDA0C2C1AD90C3CA4B2131918
:1061E00040880093230002F086FE431E9841013050
:1061F0007B06DB0F6B703F23013C1F40A4B228706D
:10620000AF70AC80002C07D0B3680133AB600021C5
:106210000800FEBD0020EBE7AC60F8E70B780370E8
:106220004B8843704B881B0A83700B79C370042022
:1062300070470420022B06D10020537811781B02EE
:10624000009A0B43138070470B8803700B881B0A5E
:106250004370022070470420009983420AD153788A
:1062600010781B0203430B80D37890781B02034302
:1062700000204B807047F8B50D004B7801240021B9
:10628000461C03702B788B4201D82000F8BD6B7838
:10629000B01C4F1C012B10D1890069184B880222B9
:1062A00033704B88B9001B0A7370691805F0D8FC6D
:1062B00004360434A4B2F9B2E4E7122359436B184C
:1062C0005A88043132705B8810221B0A7370691877
:1062D00005F0C6FC12361234ECE770B5049D1400CC
:1062E0001E00052B01D8042070BD637812781B02B4
:1062F00013432B80E378A2781B02134302226B80A6
:106300002A71211D681D063E05F0AAFCB2B22A8141
:10631000F02AE8D82800A11D0A3005F0A1FC0020D1
:10632000E2E7002310B50A789A4201D8900010BD28
:106330009A008A185488013304705488DBB2240A06
:106340004470948884709288120AC2700430EAE71C
:1063500010B51100029C062B04D004201022142B2F
:1063600001D010BD022222714B7808781B02034332
:106370002380CB7888781B02034363800431601D3F
:1063800005F06EFC0020ECE710B50C788B7804313A
:106390005C43E4B203702200013005F061FC601C34
:1063A00010BD0420022B06D10020537811781B0267
:1063B000009A0B431380704710B50C000A88023115
:1063C00005F04EFC208810BD70B504000D00049847
:1063D0001100012B01D8042070BD167852781202EA
:1063E000324302800200F83255701470E825002C08
:1063F00000D10C35023B9AB24280AA42EBD802315E
:10640000043005F02DFC0020E6E7042000998342CB
:106410000AD1537810781B0203430B80D37890780D
:106420001B02034300204B80704710B50C000A8804
:10643000023105F015FC208810BD000070B5012167
:106440001E000420049C0E400B4218D1CB40DDB24C
:106450008D4214D90A49DBB2098899420FD323002F
:10646000F6331D703300580011184978165C090284
:10647000314301332152D9B28D42F4D8002070BD8E
:10648000C845FF1F10B50C000A88023105F0E8FB73
:10649000208810BD10B50C788B7804315C43E4B2D1
:1064A00003702200013005F0DBFB601C10BD10B54D
:1064B00011000298032B01D8042010BD14785278E3
:1064C000043B120222430280CA788C7812022243D3
:1064D00042809AB28280F22AEED80431063005F06A
:1064E000BFFB0020E9E710B50C000B8803700B8898
:1064F0001B0A43704B8883704B881B0AC3708A88C1
:106500000430063105F0ACFBA088043080B210BD29
:106510000420012B03D100201378009A13707047D8
:1065200010B50C000B8803700B881B0A43704A8857
:106530000230043105F094FB6088023080B210BD57
:10654000F0B589B003931E4B029242000700D05A67
:10655000019102F020F81325061E2DD0029B012484
:106560000370019B002B04D0001903999847001970
:1065700084B26B461B7A5BB2002B0FDA1021380015
:1065800002F01CFB1925002813D130003219E1B2AA
:1065900002F066FC051E0CD10C34A4B2042304AA3C
:1065A000380005A993800696948101F0AFFD051E81
:1065B00002D0300005F0BCFB280009B0F0BDC04699
:1065C0008467FF1F70B505000C0000280CD0002068
:1065D000814209D010222000044905F041FB01202E
:1065E0002B7823736B78637370BDC0465CC0001159
:1065F000F0B506000D0017001C0085B002291BD065
:106600000020102907D1022B07D0102B03D115E051
:106610000020102C08D005B0F0BD69463800FFF707
:10662000D1FF2A0069460BE069463000FFF7CAFF38
:1066300022006946380004E0022BE9D12A00390023
:10664000300005F005F9E6E7031CF72800D9F72329
:10665000032008499AB2013A0B80D3170340064938
:106660009B189B100B80D30F04499B185B100B8069
:106670007047C046CC45FF1FCA45FF1FC845FF1FD6
:10668000034B1B888B4202D3024B4000C152704720
:10669000CC45FF1F8467FF1F014B4000185A70470D
:1066A0008467FF1F1722014B1A8070478467FF1F02
:1066B00070B505000E2005F08BF9041E13D0D02311
:1066C000037000230622837007494570033005F0EC
:1066D000C7FA064B2100DA8A62811B7E2373044BC2
:1066E000187805F0DDF870BDA067FF1F9067FF1FE9
:1066F0001C46FF1F262803D8024B4000C05A704793
:106700000148FCE7CE45FF1FFFFF000070B5060003
:106710000C00094D1C220021280005F039F9074B17
:106720001E70074B1C7005F00BFB0123002801D0E5
:10673000002312202B7070BD9067FF1F1C46FF1FA7
:10674000B167FF1F70B505000D4C0800E260A16045
:1067500010220021656005F013FB012803D11021F0
:10676000A06802F058FD10220021280005F008FB67
:10677000012803D11021606802F04DFD70BDC046B4
:106780009067FF1F70B5041E05D1002903D00622B3
:106790000D4805F065FA0D4B1D78012D11D1002C27
:1067A00005D102221A7005F043FA280070BD0022BC
:1067B0001A70074B1B78FF2BF7D02000FFF778FFEC
:1067C000F3E70025F1E7C046A067FF1F9067FF1FB2
:1067D0001C46FF1F030010B5002801D1002010BD8A
:1067E00000780B4A002803D15988D1821B7913768F
:1067F0001378022BF2D10023984200D10333137097
:10680000044B1B78FF2B01D0FFF752FF0120E6E776
:106810009067FF1F1C46FF1F002911D000280CD0D5
:106820004B79012803D140225242134303E03F2217
:106830001340032802D001204B7170474022F4E737
:106840000800FAE770B5094D0100287800280BD040
:10685000074C0622200005F003FA21002878FFF7F4
:10686000DBFF200005F074F970BDC046B067FF1F64
:106870008A67FF1F00290AD0012808D13F224B79DF
:106880009343C02B03D0403B5A425341981C70475E
:1068900070B5174D06002B78FF2B15D00A2005F098
:1068A00097F8041E10D0D0230370C83B8370114B9F
:1068B00011491B784670C3700622043005F0D0F9E8
:1068C0002100287804F0ECFF0C4B1B78012B0DD134
:1068D0000B4B1B68002B03D09B68002B00D0984704
:1068E000084B04211878084A05F0CAF870BDC04664
:1068F0001C46FF1FB067FF1F8A67FF1FAC67FF1FA3
:10690000D867FF1FDC67FF1F60EA0000014B986833
:106910007047C0469067FF1F014BDB6818687047DF
:106920009067FF1F074B10B5DA68136801331360D7
:10693000054B1878FF2803D08021C90105F0B0F875
:1069400010BDC0469067FF1F1C46FF1FF7B50E0025
:1069500002F0C8F8051E1CD00E4B06621F78002FEF
:1069600000D10778AB791020019305F031F8041EAF
:106970000FD0D0230380C73B8370019BE91DC370F8
:106980000622043005F06CF921003800E66004F0BE
:1069900087FFF7BD1A46FF1F014B18787047C046A6
:1069A000B067FF1F054B002805D1054B1A78054B32
:1069B000002A00D1014B18007047C046A067FF1F96
:1069C000B067FF1F8A67FF1F014B58687047C046BA
:1069D0009067FF1F024B1868431E9841C0B2704772
:1069E000B467FF1F421E03000120152A03D9FF3B95
:1069F0005A425341D8B27047F0B51C0000230E0034
:106A000085B0039002920B70029A934201D300204A
:106A100019E0E55C5A1CD2B2002DF8D00298511949
:106A20008142F4DC0233DFB2A35C18000193FFF76C
:106A3000D9FF002807D0013D019A0399EBB23370CA
:106A40008A4202D1E01905B0F0BDDB19DBB2DBE709
:106A500010B50C0002F09EF803001220002B03D0AA
:106A60002100588805F014F910BD000070B50E4DD6
:106A700084006359002B15D0186A002801D005F056
:106A80002FF82B59586A002801D005F029F82B5906
:106A9000986A002801D005F023F8285905F020F85D
:106AA00000232B5170BDC046C067FF1F1C4B70B543
:106AB00004000E00150099420AD11A4B1B68002BE6
:106AC00001D1122070BD1B68002BFAD09847F9E75E
:106AD000154B994215D1134B1B68002B0AD01B682C
:106AE000002B07D09847002804D1104B1C70104B86
:106AF0001D70E7E729002000FFF7AAFF0028E1D179
:106B0000F3E7080001F0EEFF0028DAD00378032055
:106B1000A342D7D12900300005F0BAF8D2E7C04629
:106B2000FEFF0000BC67FF1FFFFF0000B967FF1FEB
:106B3000B867FF1FF7B50400808801F0D3FF002578
:106B4000A84203D00578A08802F008F81C4E3378DC
:106B5000002B1FD0AB421DD11A4B28001978FFF72C
:106B600077FF002818D000233370A3790820A77876
:106B7000A688019304F02CFF011E0DD0D0230370D2
:106B8000CA3B8370019B477086808371280004F0A4
:106B900087FE01E0002DE8D1A0880B4B8200D3587E
:106BA000002B01D0FFF762FF1721A088FFF768FDD7
:106BB000A08801F027FDA08801F0FEFDF7BDC046CA
:106BC000B967FF1FB867FF1FC067FF1FF0B587B029
:106BD0001D000CAB1B88070001930DAB1B88142014
:106BE00002930EAB1B88160003930FAB1B8800911A
:106BF000049310AB1B88059304F0EAFE041E1AD020
:106C0000D0230370CB3B47708370C67006222900E7
:106C10000430002D11D005F023F8019B2100638181
:106C2000029B0098A381039BE381049B2382059B25
:106C3000A37404F035FE07B0F0BD04F0A9FEECE744
:106C4000F7B5009308AB1B8807000C200D00160059
:106C5000019304F0BDFE041E13D0280001F042FF92
:106C600000280FD00078D0232370C93BA370009B6D
:106C700021002381019B6770A580E680638104F079
:106C80000FFEF7BD014B1878EDE7C0461C46FF1F0D
:106C900013B5040064890389C2888188C078009490
:106CA000FFF7CEFF13BD000010B5044C206800288C
:106CB00003D004F015FF0023236010BDC467FF1F3D
:106CC000A122F0B5818892004A43384B384F1B68A7
:106CD00004009B189D2292009B18827989B01A604B
:106CE0003B68002B5FD01D78324B1B68002B04D013
:106CF0005B68002B01D00020984726000836310041
:106D0000E079FFF7B7FD237DE0710200E07804939E
:106D1000638A29000393238A0293E3890193A3885A
:106D200000933300FFF752FFE378002B0BD1E28989
:106D3000A379A18802920196E279280000920122AB
:106D400001F0DAFEE0703B68002B20D0FFF7ACFFCB
:106D5000194D287800281AD0184B1978FFF778FEBB
:106D6000002814D02B78E67808200793A78804F031
:106D70002FFE011E09D0D0230370CA3B46708370DA
:106D800087808671079804F08BFD00232B701721F4
:106D9000A088FFF775FCA08801F034FCA08801F002
:106DA0000BFD09B0F0BD064B9DE7C0463409FF1F3F
:106DB000C467FF1FD867FF1FB967FF1FB867FF1FB2
:106DC0001C46FF1FF8B5070008000E0001F08AFE00
:106DD000041E18D02620FFF78DFC051E00D1257853
:106DE000062004F0F5FD041E0DD00021062204F05B
:106DF000CFFDD0232370C23B21006770A370A68013
:106E0000E8B204F04DFDF8BDF0B585B001930AABD2
:106E10001B78070002930BAB1B7808000D00009253
:106E2000039301F05FFE061E22D0102004F0D0FD77
:106E3000041E1DD01022002104F0AAFD2620FFF719
:106E400059FC002800D13078D0232370C13BA370B7
:106E5000009B21002372019B67706372029BA580D7
:106E6000A372039BC0B2E3720C9BE36004F018FDB5
:106E700005B0F0BDF7B50D00019001F033FE071E1F
:106E800020D00E2004F0A4FD041E1BD02620FFF706
:106E900031FC061E00D13E78D0232380C53B06225C
:106EA000A370F91DE01C04F0DBFE019B2A00638146
:106EB0000123DD401A401D40210022736573F0B2AA
:106EC00004F0EEFCF7BD0000F0B585B002901000B4
:106ED0000D0017000A9E039301F004FE041E31D03A
:106EE000029B002B2ED1039B02795B0724D5122332
:106EF00013430422002E08D10B99002905D10C99C7
:106F0000002902D10D9900291AD01A430D9B227134
:106F1000002B00D0C9E0002E00D1CFE0002D00D022
:106F2000CCE0606A002801D004F0DAFD1C213000BA
:106F300004F02EFE606205E002239A430E33D7E789
:106F400093432371654BBA00D458002C00D1AAE0BA
:106F5000002E10D0236A002B03D11C2004F058FE11
:106F600020625E4BBA00D358186A002803D01C2256
:106F7000310004F075FE0C9B002B12D0574CBB0067
:106F80001D596B6A002B03D1162004F041FE686284
:106F9000BB00E358586A002803D016220C9904F06D
:106FA0005FFE0D9B002B11D04C4DBC006659B36A9F
:106FB000002B03D1142004F02BFEB0622B59986AE9
:106FC000002803D014220D9904F04AFE380001F085
:106FD00089FD051E67D0414BBA00D358002B62D003
:106FE0001A6A3420002A00D11C389A6A002A01D07B
:106FF000143080B20B9A002A01D01C3080B25B6A38
:10700000002B01D0163080B204F0E2FC041E4AD0FE
:107010001822002104F0BCFC2620FFF76BFB019036
:10702000002801D12B780193D0232370029B2000EC
:1070300063700A23294EA370039BBD00A371AB5953
:10704000A780196A1830002905D01C22A06004F01E
:1070500007FE200034307359996A002907D00300D5
:1070600014221433E060029304F0FAFD02980B9BA3
:10707000002B08D003001C221C330B9920610293C3
:1070800004F0EEFD02987359596A002903D01622C4
:10709000606104F0E5FD6B462100187904F000FC06
:1070A0003800FFF7E3FC05B0F0BD10220D9B0D99F1
:1070B0001B69A018236204F0D3FD2CE70B9B002B67
:1070C00000D13FE7012D00D03CE7606A002801D0E5
:1070D00004F006FD1C210B982AE7C046C067FF1F7D
:1070E00010B5044C2068002803D004F0F9FC0023FC
:1070F000236010BDB467FF1F0B4B07B51A68002A49
:1071000001D100200EBD6946531C012012780731C1
:10711000FFF772FC0028F4D0027801231000184019
:107120001A42EED0EEE7C046D067FF1FF0B51F4F02
:1071300001203B6887B0002B25D09B78059300F099
:10714000B3FB002821D00A20FFF7D4FA04000B205B
:10715000FFF7D0FA164B05001E78731E9E413B6860
:10716000F6B2191DD878FFF757FB3B682900DA7A89
:10717000043303929A790193029200903300200025
:10718000059A04F0E5FD07B0F0BDFFF7B5FF002854
:1071900005D00620FFF7AEFA04000720D8E7082044
:1071A000FFF7A8FA04000920D2E7C046B467FF1F22
:1071B000B067FF1F70B50A4E040033780D00FF2B37
:1071C0000DD0042004F004FC011E08D0D02303706D
:1071D000CE3B45708370C470307804F061FB70BDA5
:1071E0002C46FF1F70B5040006200D0004F0F0FBD4
:1071F000011E0AD0D0230370CD3B8370054B447031
:107200001B688580187804F04BFB002C01D0FFF739
:1072100067FF70BDB467FF1FF8B5264F06003B68D7
:107220000D001124002B05D10522234B1B7813429E
:1072300002D112242000F8BD204A10241268002A2E
:10724000F8D01278002AF5D0DB0719D52B789A1ED2
:10725000012A1AD80C2004F0DBFC13243860002823
:10726000E8D000230A22437029000670023004F09F
:10727000F7FCFFF75BFF041E0AD0FFF731FFD9E7E9
:1072800000F012FB0028E1D1E4E7002BE2D0D0E7C8
:107290000B4B1B78032BCDD11D20FFF72BFA094B8D
:1072A00018800028C6D0084B04211878074A04F03B
:1072B000E7FBBFE7B467FF1FB167FF1FD067FF1F82
:1072C000B067FF1FAE67FF1FDC67FF1F60EA0000AB
:1072D000F7B50193194B14001A78052306000F0027
:1072E00012201A4221D0012920D1154B1D68002DF2
:1072F0001BD002201F2C18D8002C02D0019B002B81
:1073000013D0104B1F221E706E1C0021300004F0A1
:107310003FFB01992200300004F0A2FC3100200064
:107320002C70002F06D004F083FAFEBD064B12200D
:107330001D68DCE704F0CCFBF7E7C046B167FF1F30
:10734000D067FF1F2C46FF1FCC67FF1FF8B50F4EFD
:1073500012243368002B17D01B780F3C834213D1C3
:1073600000250B4F0221387804F03AFB094B042129
:1073700038781D8004F034FB074B28001D803368EB
:107380005C7004F01DFC04002000F8BDB467FF1F12
:10739000DC67FF1FC867FF1FAE67FF1F70B50128BE
:1073A00023D11B4C2388002B03D01A4A1578002DBB
:1073B00007D0194B1B68002B02D01878FFF7C6FFC7
:1073C00070BD3B2B02D93C3B2380F9E7134E0221D1
:1073D000307804F005FBFA222388920002215A43F8
:1073E000307804F00DFB2580EAE70B4B1B68002B7F
:1073F000E6D00B4B1B785B07E2D5084B02211878CF
:1074000004F0EEFA0022024B1A80FFF769FED7E77C
:10741000C867FF1FAC67FF1FB467FF1FDC67FF1F54
:10742000B167FF1FF8B51E4D2868002803D004F08F
:1074300057FB00232B601B4E3068002803D004F05C
:107440004FFB00233360184F05243B781800204081
:10745000234221D0154800F02BFA3B78234213D069
:10746000202004F0D5FB2860002813D02022002122
:1074700004F08EFA202004F0CBFB041E306005D00F
:107480002022002104F084FA002004E0286804F09F
:1074900027FB2C601320F8BD00F00AFAF4E7C04681
:1074A000D067FF1FCC67FF1FB167FF1F2046FF1F7C
:1074B00010B50A4C23681A1E0ED0002808D10130DE
:1074C000587004F07DFB002805D02368002B02D003
:1074D0000021FFF787FE0122100010BDB467FF1FD7
:1074E000F7B5274E050033680191181E21D05C784E
:1074F000244F012C30D1FFF7FFFD002825D02000BC
:10750000FFF7F8F80400412814D91F4B022118781E
:107510001E4A04F0B5FA1E4B3C3C1C800222336824
:107520005A703B78002B14D128000199FFF75AFEBE
:107530000120FEBDFA2292004243002AEED0124BF7
:107540000221187804F05CFAE8E7FFF7D3F80200AC
:10755000F3E700233B70EBE73B78002BE8D10320F7
:1075600004F036FA011E08D0D0230370CC3B4570DE
:1075700083703368187804F093F9FFF7B1FDD7E70B
:10758000B467FF1FAC67FF1FDC67FF1F60EA0000E6
:10759000C867FF1F10B51749838802008B4220D0AF
:1075A00011D815498B4217D0144900205B1899B2A5
:1075B000012907D8926811785A425341D8B2FFF78F
:1075C000F9FD012010BD0E4A00209B1807229BB236
:1075D0009A424041C0B2F5E783681878FFF768FF28
:1075E000F0E7836899785A78090218781143FFF711
:1075F00077FFE7E70A20000006200000F8DFFFFF22
:10760000AFDFFFFF014B18707047C0462D46FF1FCC
:1076100010B5064C207001F041FA207804F040FBD0
:107620000521207800F062FD10BDC046DC67FF1F19
:107630000BB273B50D00002B00DBC4E0884B18784B
:1076400004F0B6FB041E0ED00378912B0FD0A22BB2
:1076500000D1A1E0834B1878FF2852D0210004F01C
:107660001FF900284DD180200002684076BD437884
:107670000F2B76D013D8052B70D00E2BEAD1808833
:10768000794B98422BD8794B98421BD8784B98422B
:10769000E0D1A3681878591CFFF774F838E03E2B46
:1076A000D8D18378032B74D06CD8012B6ED0022BE9
:1076B000D0D1704B1B68002B23D05B68002B20D0EF
:1076C00098471EE06C4BC0180C28C3D804F090FA01
:1076D0001DC2C2150BC20B0B0B3223C23C00674B01
:1076E000C0180728B6D8664B1B68002B09D01B684A
:1076F000002B06D0200098470AE0A3681878FFF70F
:10770000C7F8200004F03CFAADE7A068FFF762F884
:1077100000289FD0F5E7A3681B78002BF1D0554BCC
:107720001B68002BEDD01B68002BEAD021005548C8
:107730009847EDE74F4B1B68002BE2D01B68002BEE
:10774000DFD021005048F3E7504B1B68002BD8D006
:107750005B68002BD5D021004348E9E7FFF7EAF941
:10776000CFE780884A4B984203D04A4B984200D0DA
:1077700070E7464B1B68002BC3D05B68002BC0D062
:107780002100D5E7153B012BBBD963E7FFF798FA3A
:10779000B7E7FFF77DFAB4E73F4B1B78042B07D11F
:1077A00000236A4613800179408800F0C5FCA8E7F1
:1077B000364B1B68002BA4D05B68002BA1D00100C6
:1077C000364898479DE7012421420AD0294B1B687F
:1077D000002B04D05B68002B01D0002098470120CB
:1077E00043E78B070AD5264B1B68002B04D05B6848
:1077F000002B01D020009847022036E70421280002
:1078000008400D4200D131E7254E3388002B21D0AE
:10781000013B9BB23380002B1AD1FFF7DBF8002825
:107820000AD0204B1C70164B1B68002B04D05B68E1
:10783000002B01D020009847FFF7C6F8694601F0F9
:1078400001FD6846FEF7FEFF1D20FEF753FF308066
:1078500004200AE7024B187804F0C2F8F8E7C046A3
:10786000DC67FF1F2D46FF1F0E20000001200000D7
:1078700009100000D467FF1FFEDFFFFFAFDFFFFF2F
:10788000D867FF1F0C2000000B200000BC67FF1F03
:107890000D20000013200000B167FF1FFFFF000054
:1078A000AE67FF1FAC67FF1F10B501F09BF910BD5D
:1078B000014B18607047C046D867FF1F0B88002037
:1078C000162B01D817230420014A13807047C046A5
:1078D0008667FF1F00207047074A03001188814216
:1078E00007D091880020994202D101308000101801
:1078F00070470020FAE7C046E467FF1FF0B58F78B5
:1079000006000D00C7B01E2F15D1FFF7E5FF051EBD
:1079100003D10024200047B0F0BD00223B0031001D
:10792000C078009200F0B2FB0400A81C00F0D3FB6A
:10793000FF23EB70EEE7264B062403931B78FF2B07
:10794000E8D0182FE6D87B08224A013BDB000292E0
:107950009A589446002ADDD0029AD3185B68002B0F
:10796000D8D00878002802D14B78012B02D1062408
:10797000122FCFD107AFAB88697800976446AA6809
:10798000A047041EC6D1AB78029A5B08013BDB001E
:10799000D318390030005B689847041E0BD1AB78D0
:1079A000042BB6D0039A310010782200009700F023
:1079B0006DFB0400AEE76A78002AABD1AA7805A96E
:1079C0003B88087130000A704B80FEF747FBA0E748
:1079D0003046FF1F6CC000111D4B37B505009842A3
:1079E0000BD000290AD1FFF777FF002805D11948ED
:1079F000FFF772FF002800D0058037BD01291AD19A
:107A0000FFF76AFF041EF8D001235B420380A378CE
:107A1000FF2BF2D0FE2B07D00023E0781422009336
:107A200029001E3300F032FBA01C00F054FB0123A0
:107A30005B426380E1E70229DFD1013901F0BEF842
:107A40000028DAD12800FFF747FF041EDFD1D4E772
:107A5000FEFF0000FFFF0000022210B5074B52425C
:107A60001A80074801325A809A80DA8000F07EFA44
:107A7000044801F025F8002010BDC046E467FF1F50
:107A8000FD780011D97900110388F7B50400002BA7
:107A900002D102252800FEBD426802211378254844
:107AA0005268FEF7A5FD00282ED0234F01253A8805
:107AB000002AEFD0802321885B0201259B1A99427E
:107AC000E8DC0C2004F0A4F8061E31D03B882288A4
:107AD0009C4600231800019561469DB2491989B260
:107AE000AA421BD8002801D062443A80002330000B
:107AF000082208C0210004F0B3F8104A1368002BD4
:107B000013D100251660C5E76268022113780C487E
:107B10005268FEF76DFD0028C7D1BAE760681D0105
:107B20004019418101330198D6E71A001B68E6E746
:107B30001325AFE7DAC000112E46FF1FE067FF1FD5
:107B4000D8C00011014B18707047C0463046FF1F67
:107B500014230A0010B51A40194204D00122102142
:107B600001F048F810BD4B06F9D4012088434000CD
:107B7000F8E710B514008B0604D50122102101F09E
:107B800039F810BD08230A001A40194202D14BB23D
:107B9000002B0FDA102101F02DF8002808D0230067
:107BA000F9331B78002BECD0F8342378012BE8D183
:107BB0000020E6E703208907FAD4E2E7F0B51F00CA
:107BC000184B85B01C68019002910392002C27D1BC
:107BD000200005B0F0BDA5683301ED186B89019A4E
:107BE000934211D3029A93420ED8002F04D10A9BDC
:107BF000002B10D12C00EBE73B002978039A686832
:107C0000FEF7F6FC0028F2D10136B6B2A388B342E3
:107C1000E1D82468DAE7A3680A9A5B891380E9E768
:107C20000026F3E7E067FF1F37B50C000A88498894
:107C30000123914217D3002A15D0651D23792A000C
:107C400002210A48FEF7D4FC102300280BD0237928
:107C50006188208800242A000094FFF7AFFF0A23E0
:107C6000A04200D0230018003EBDC046DAC000117B
:107C700013B50A0008884988012388420BD80028D8
:107C800009D00024137905320094FFF797FF0A23E7
:107C9000A04200D02300180016BD13B50A000888C2
:107CA0004988012388420BD8002809D00024137981
:107CB00005320094FFF782FF0A23A04200D0230080
:107CC000180016BDF0B58BB003904A8808880E00E6
:107CD0000123824255D3002853D00023012704AC4E
:107CE00023700022718813000092FFF767FF051EC2
:107CF0003ED02078002835D12B78022B18D1677020
:107D00006A8983000130E31880005A806968022282
:107D1000201803F0A5FF23780133DBB22370042B76
:107D200019D93B006889013080B2002BD9D01FE0FF
:107D300002236370122358436A89231804305A803F
:107D400069681022201803F08BFF23780133DBB21F
:107D50002370002BE5D10C4A6B899B185A42534182
:107D6000DBB2DFE76378012BE4D12B78022BC7D09D
:107D700022780A23002A04D021000398FEF798F9FC
:107D8000002318000BB0F0BD0100FFFF0F4BF0B552
:107D900004001868002816D083685D89A54207D8BA
:107DA0008288AE18B44203DA12019A18934201D1C4
:107DB0000068EFE71E005F891036A74204D1002952
:107DC00000D00D801800F0BD3300EFE7E067FF1F23
:107DD00070B505000C0008880021FFF7D7FF0300ED
:107DE0000120002B04D022002800197AFFF7C1FEE1
:107DF00070BDF7B50C00002501902300F6331B7809
:107E0000AB4201D800200AE06B00E65A00213000A6
:107E1000E718FFF7BBFF002802D126800130FEBD26
:107E2000017A0198FFF794FE002802D03B88238056
:107E3000F5E70135EDB2E0E710B504000888002150
:107E4000FFF7A4FF03000120002B03D02000197AC4
:107E5000FFF77EFE10BD0000054B1B68002B01D113
:107E6000180004E09A6852898242F6D198887047D7
:107E7000E067FF1FF0B50E27002687B0039302AB23
:107E8000FF183E8005001F4B40891400984207D020
:107E90002B78013000976A6880B2FFF78FFE0600EA
:107EA00002212B7818486A68FEF7A2FB00280FD041
:107EB0006C892000FFF7D0FF002802D0013C041994
:107EC000A4B2039B002B00D01C80300007B0F0BD93
:107ED00002212B780D486A68FEF78AFB0028E7D15B
:107EE00002212B780A486A68FEF782FB002807D037
:107EF000002EDED03B88A342DBD17489013CDFE752
:107F00006C89DEE7FFFF0000DAC00011D8C0001165
:107F1000D6C0001110B50C00FFF7DEFC03000220F4
:107F2000002B0AD0002C00D023609B781720FE2B5A
:107F300003D00138FF2B00D1002010BD73B50D0018
:107F400001A904001600FFF7E5FF172805D0002E51
:107F500004D129002000FEF727F976BD0122102167
:107F6000200000F047FE0028F3D0F6E7014B186030
:107F70007047C046F067FF1F37B56B469D1D010077
:107F800004000222280003F0CBFC2B88B02B0ED17A
:107F90002379122B09D12300FF339B78012B06D1C3
:107FA0000121608800F0E0F801E01B2BF8D037BD1C
:107FB00010B5054B0421187000F098F8FFF74CFD40
:107FC000FEF770FB10BDC046F467FF1F0020F0B540
:107FD0000BB20F0087B0834234DA274B187803F0D6
:107FE000E7FE051E2BD00378A02B25D103AE310070
:107FF000FEF7E4F8041E0BD1B378DB0724D51F4B42
:1080000006341B68002B03D03100688898470400B1
:10801000A868002801D003F08BFE002C08D1184A74
:10802000039B1340174A934206D0B3781B2B03D00F
:108030000121688800F098F8280003F0A1FD802055
:108040000002784007B0F0BD0F4B1B68002B10D02A
:10805000310068889847041EDAD07378002BD7D196
:10806000B27801A90A704B800C716888FDF7F6FFA1
:10807000CEE70624F1E7C046F467FF1FEC67FF1F59
:1080800000FFFF0000011200F067FF1FF7B501902D
:10809000822040000D0017001E0003F099FC040030
:1080A0001320002C12D0B02320002370089BFC2248
:1080B0006770658026710830002B08D0190003F026
:1080C000CFFD2100019803F0EBFB0020FEBD0899D5
:1080D00003F05EFCF5E710B5041E06D00078FD281D
:1080E00003D803F04DFCFF23237010BD0A1F93B289
:1080F00010B504000220032B05D882400020024B5B
:10810000D1529B189C7010BD1468FF1F0B8870B56E
:10811000043B04000D000220032B0BD8012120009A
:1081200000F04CFD03001420002B03D02900200098
:1081300000F0DEFB70BD000007B51300034A00929B
:108140000A00012100F02CFC0EBDC0467583001111
:1081500007B5019203220092024B0A00122100F09F
:1081600049FC0EBDF383001107B56B4601AA1180CF
:108170000449D88008780633012802D1190003F099
:108180002FFB07BDF567FF1F0C4B10B518700023C0
:10819000FF210B4A1380138193819380094A5380F6
:1081A0001370517293819372D174D3821375517786
:1081B00003F006FE00F0FCF910BDC0462468FF1F66
:1081C0001468FF1FF667FF1FF0B58DB06B460020E7
:1081D00003910C229B5E834200DBB0E05D4B18787C
:1081E00003F0E6FD051E00D1A4E00378902B00D03B
:1081F0009DE006AF01004688380000F013FA796868
:108200000400002900D19CE03B88052B6ED13B89FE
:10821000032B1CD905AC200000F0A2F86288172AB5
:1082200061D83989131D994231D179682378043195
:108230000291D90738D5607800F08EF9071E06D074
:10824000002303712378012B08D0132B23D0A868B7
:10825000002800D178E003F06BFD75E06288029998
:1082600009A800F0A6F80290380000F08BF909AADE
:108270002378387A0192002231000092029A00F0AD
:1082800012F9380000F064F9029B002BDFD03000B7
:1082900000F080F9DBE70378032BD8D162880299DC
:1082A00009A800F0D6F8DEE7122B13D1029909A82D
:1082B00000F0B5F8021EEAD127498B88002BC6D002
:1082C000887909A92378019161780091310000F043
:1082D000EAF8BCE7002302AA93833000617809AA78
:1082E000FFF72AFFB3E71D4B0993F6E7042B02D0F3
:1082F0009A1F012AABD8184A043B9B00995A0029BF
:10830000A5D0D218907831003A0000F0AEF80028DD
:108310009DD13B88042B03D001213000FFF724FFBF
:10832000012C04D1A868002801D003F001FD280029
:1083300003F026FC8020039B0002434018000DB090
:10834000F0BD012800D182E701213000FFF70CFFCA
:10835000EDE7C0462468FF1F1468FF1F01001700E7
:108360000B7803704B784370CB788A781B021343E9
:10837000438070470A88030002700A88120A42701C
:108380000A88012A06D14A8882704A88120AC27075
:108390000420704702208242FBD14A8804309A7040
:1083A0004A88120ADA708A881A718A88120A5A71FF
:1083B000EFE710B50400012082420CD94B780A780F
:1083C0001B0213432380834206D1CB788A781B0299
:1083D00013436380002010BD022BFBD1CB788A7839
:1083E0001B02134363804B790A791B021343A3805A
:1083F000F0E70B8803700B881B0A43704B8883706F
:108400004B881B0AC3708B8803718B881B0A4371CE
:10841000CB888371CB881B0AC37108207047030087
:108420000120082A14D14A780878120202431A80DF
:10843000CA788878120202435A804A79087912026F
:1084400002439A80CA798879120202430020DA80B6
:10845000704710B504000120022A05D100204B7896
:108460000A781B021343238010BDF8B506001020C4
:108470000F00150003F0ACFA04000120002C0ED010
:10848000A0230C22290023806780201D002D07D007
:1084900003F0E6FB2100300003F002FA0020F8BDF3
:1084A00003F076FAF6E7F7B51E00009008AB14204B
:1084B00017001D78019103F08BFA041E12D0A2233D
:1084C0000370019B47704380099B057146710C2224
:1084D0000830002B07D0190003F0C2FB21000098E0
:1084E00003F0DEF9F7BD099903F052FAF6E737B564
:1084F000041E0FD04388002B0CD00025C188132305
:10850000007A172201950095FFF7CDFFFF236580C4
:108510006372257037BD000010B50C4904004A880D
:10852000002A09D08B89002B05D00020CB8A02229B
:10853000834201D010BD012213000A2043430020D2
:108540004032C854C81842800472F3E7F667FF1F30
:108550000023438003707047094B00211A0010B5B7
:108560005C88002C06D01C79844203D10A234B433B
:10857000D01810BD01310A330329F1D10020F8E7EA
:10858000F667FF1F10B50400407A03F0F9F9FF23E6
:10859000637210BD7047043010B580B203F068FA02
:1085A000002803D00421494203F04AF910BD00001D
:1085B00070B50025104CA0682580A581A580A84233
:1085C00002D003F0B5FBA56000250C4C0C4B606D90
:1085D0001D80230058331D70A84202D003F0A8FB71
:1085E000656500256068002801D003F0A1FB013516
:1085F00008340A2DF6D170BDBC68FF1F6068FF1FEC
:10860000B068FF1F70B5041E09D1054D2880A881F0
:10861000A880A868002802D003F08AFBAC6070BD77
:10862000BC68FF1FF0B54B8885B001930023436001
:108630000A7905000F00022A00D07BE0CA88032ACD
:1086400017D98B685E7819783602DC78D8790E43B2
:1086500099781B7A24021B020C43034353495BBAEB
:108660000B80331D93421ED1042C04D0631F022BB8
:108670000ED9012015E0019A4D4B1201D35A002B5F
:1086800006D00198FFF7BEFF4A4A13690133136110
:108690000421B8682E812C80494203F0D1F868602B
:1086A000002005B0F0BD434D042C06D0631F022B03
:1086B0000FD9EB680133EB60DBE7019A3C4B120109
:1086C000D35A002B05D00198FFF79CFF2B6901338B
:1086D0002B61374B30000293019B029A1B010193DF
:1086E000002301998C468B52130063449C800393B2
:1086F0009E81FFF750FF039B041E986016D0042153
:10870000B868494203F09CF8FA880100043A200056
:1087100003F0A6FA0199029AFB888A5A043B9B1837
:10872000029A8B522B6801332B60A2E7AB690133AD
:10873000AB619EE71E4B0293019B1E01029BF35A05
:10874000002B2DD002998C19A068002828D0012A6E
:1087500026D1FA889B189BB27352A189994217D3EC
:108760009B1AC018B96803F07BFA029BA289F35ADE
:10877000934200D07DE700222B81A3882B80A36841
:108780006B60029BF2520B4A53680133536070E7EF
:10879000084A9368013393600198FFF733FF68E755
:1087A000044A536901335361F6E7C0462668FF1F48
:1087B000BC68FF1F2C68FF1F70B5051E15D10B4C40
:1087C0000B4B1880230058331870606D002802D0BE
:1087D00003F0AEFA6565250050356068002801D0C9
:1087E00003F0A6FA0834AC42F7D170BD6068FF1FF1
:1087F000B068FF1FF0B51700A12285B09200019369
:108800004243394B06001B680C009B18D933FF33D9
:108810001D78FDF741FF0430854204DD3000FDF78F
:108820003BFF0430C5B2BD4207D33A0000213000FF
:10883000019B03F095FA05B0F0BD2900380003F064
:1088400067F92300C6B250331E700393019B2900C1
:108850006365380003F074F9CBB20293002B02D0A9
:10886000039B01361E7000262300503303931B78B0
:10887000B34204D8606D002831D10020DBE7029AB2
:108880002800002A04D0013B1000B34200D0280089
:10889000F700E719387003F09BFA786000280ED0D3
:1088A0003A78019903F0DCF9019A3B780136D31844
:1088B0000E4A0193D369F6B20133D361D4E7039B27
:1088C00018706065A74205D1084A1320D36A0133A6
:1088D000D362B0E7606803F02BFA0834F2E703F0E4
:1088E00027FA00236365C8E73409FF1F2C68FF1FC0
:1088F000F7B50D0007000421686802F0A1FF2B897D
:10890000040003702B891B0A43702B8883702B880B
:108910001B0AC3702E8902250436F6B2FB2E15D829
:108920001B4B9F4214D10C2003F052F81135011E4D
:108930000CD0902303708E3B0371043B4380154B96
:108940008460C680187802F0ABFF00252800FEBDC9
:108950005C237B43104AD3180093583301931B7850
:10896000002B0FD10300320038000099FFF742FFBF
:10897000019B05001B78002BE8D13800009903F01B
:10898000F7F8E3E7054A0725536A01335362DDE749
:10899000FEFF00002468FF1F6068FF1F2C68FF1F98
:1089A000F0B587B0009017200F0016000193FFF775
:1089B000F2FD1325041E19D00C98031E02D0019954
:1089C000201D9847030AE370052302AAA070043013
:1089D000908127700098667003A993800494FFF734
:1089E00087FF051E02D0200003F0A2F9280007B07F
:1089F000F0BD0000F0B587B01F000CAB1B780391F1
:108A0000059301210DAB06001C78049200F0D6F806
:108A10001425002821D02000FFF77EFD0135041E1B
:108A20001BD01149059B0A7803700132D2B2131E84
:108A3000C68001D101231A000B7022713000049B03
:108A400003990097FFF7ACFF051E09D12300210011
:108A50000648074A093302F0DBFF280007B0F0BDE3
:108A6000002363802370F8E72868FF1FEF8400115C
:108A700030750000F8B505000E00064C064F23685F
:108A8000002B02D03100280098470434BC42F6D1B4
:108A9000F8BDC046CC68FF1FE068FF1F0123064AEF
:108AA0005B425380002313715362044A1360536086
:108AB0009360D36013617047E068FF1FCC68FF1FAD
:108AC0000200002310B506499C000859002801D176
:108AD000625010BD0133052BF6D11320F9E7C046D3
:108AE000CC68FF1F034A5388181A4342584140423A
:108AF00010407047E068FF1FF0B585B002930AABE5
:108B00001F780CAB1B88009008000E0001920393A5
:108B1000FFF7E8FF05001120002D1BD10E48FFF7DD
:108B2000E1FF04001520002C14D006220B99A77138
:108B3000E01D03F095F8019B30002371029B290092
:108B40006371009B66802370039B6562E381FFF77E
:108B500091FF280005B0F0BDFFFF000010B5FFF742
:108B6000C1FF04000220002C12D060880121FFF711
:108B700081FF606A002801D002F0B2FF28220021A4
:108B8000200002F005FF012300205B42638020717A
:108B900010BD000030B5074A074C55880100137816
:108BA0000020A54204D05B1A59424B415842104064
:108BB00030BDC046E068FF1FFFFF0000084A10B547
:108BC00001230C00904208D0FFF78CFF031E04D055
:108BD000037923405A1E9341DBB2180010BDC046F2
:108BE000FEFF0000024B1879431E9841C0B2704747
:108BF000E068FF1F70B504000D001600FFF772FF5C
:108C0000002804D10D4B9C4200D0143070BD416A45
:108C100003790520002907D012221A40102A02D118
:108C20000520002EF2D10F20DB06EFD5897E0C2027
:108C3000A9428941494249420840E7E7FEFF000056
:108C4000030010B5002800D110BD0348034A418835
:108C50009142F9D09847F7E7E068FF1FFFFF000057
:108C6000002330B5C45CCD5C6C40D4540133102B70
:108C7000F8D130BD0F23002210B5C45C640022433C
:108C8000CA54C25CD209013BF7D210BD02000100F8
:108C900010B52032103102F0DBFE10BDF0B58BB004
:108CA0000390102005931700049102F0B1FF00908B
:108CB000102002F0ADFF009B13240190002B05D083
:108CC00000280CD11324009802F00AFF019B002B0E
:108CD00002D0180002F004FF20000BB0F0BD1020FD
:108CE00002F096FF0600102002F092FF1324050008
:108CF000002E00D1AEE0002819D01022002102F091
:108D000047FE32002900039802F0A2FE041E0ED195
:108D100033787F2B51D830000099FFF7ABFF009BD1
:108D20001B787F2B53D801990098FFF7A3FF3000E1
:108D300002F0D6FE002D02D0280002F0D1FE002C59
:108D4000C1D1102002F064FF0600102002F060FF85
:108D50000290002E7CD0002878D03A000F322300F9
:108D60000125121105D00F333B4015B25A42534131
:108D70001BB26A1E1201002B33D0049BD2B298188A
:108D80000099029AFFF76CFF013D1022002130008C
:108D900002F0FEFDADB2049F2D017D19AF4242D01D
:108DA000002C33D0300002F09BFE029B002B00D140
:108DB00089E7180002F094FE85E729003000FFF7EC
:108DC00059FF28002549009AFFF74AFFA7E7290025
:108DD0000098FFF74FFF28002049019AFFF740FF56
:108DE000A5E70F210F4004998A18D9B28F4208D9FC
:108DF000D15C06A819540133102BF6D1029A0199BF
:108E0000C0E7791A48424141C901F2E73900300010
:108E100006AAFFF725FF3200039806A902F018FE04
:108E200010370400BAE7002CBCD13000029906AA22
:108E3000FFF716FF320006A9039802F009FE082288
:108E400004003100059802F00BFFABE71324A9E7FB
:108E50001324AAE7002800D06EE733E7E0C0001132
:108E6000F0B58BB00F0016000225009000283FD00F
:108E7000002A3DD00B1DDBB21800029302F0C8FEA1
:108E80001135041E34D0FDF747FD05003A00009966
:108E9000201D02F08DFEEBB20393E3702B0CDBB2CE
:108EA0002F0A00936370FFB22B0E2370A7700193FB
:108EB000FDF72CFD1022010006A802F079FE21002A
:108EC000029A04AB06A8FFF7E9FE051E0DD1039B2D
:108ED00008223370009B04A9B370019B7770F37074
:108EE000301D02F065FEFDF71DFD200002F0F8FDCB
:108EF00028000BB0F0BDF0B58FB00D00149E0390AC
:108F000004920593002A03D1022420000FB0F0BD83
:108F1000002EF9D00398FFF7E5FD1424071EF4D0C6
:108F20007278337812021A43B3781B041343F27831
:108F300012061A43036A0192934201D30133E3D12B
:108F4000002D03D03B7901249B07DED508220021A8
:108F500006A802F01DFD059B13240433DBB21800A4
:108F6000029302F055FE051ECFD0059A04990430F5
:108F700002F01EFE04223100280002F019FE390022
:108F8000102210310AA802F013FE2900029A06AB43
:108F90000AA8FFF783FE041E0FD1082206A908A81D
:108FA00002F006FE0822311D08A802F051FC01283B
:108FB00007D101990398FDF7C9FC280002F090FD44
:108FC000A3E70124F9E7000070B51C4C05002368F5
:108FD000181E10D0002D14D11A78002A0CD1981C1C
:108FE000083202F03DFE02F013FF0135002808D1DF
:108FF00023681D70012070BD0A331800082202F09A
:109000002FFE2368002BF5D0122002F0E1FC061E93
:109010000DD0C12321680370457002311022023047
:1090200002F01EFE23683100587802F039FC2068F7
:1090300002F056FD00232360DCE7C0460869FF1FED
:10904000F8B504002020FDF755FB0D4EA700BB59D5
:109050000500002B0DD000280BD0D878FF2809D1AF
:1090600008492A000C55F35907480333611802F0E8
:10907000CFFCF8BD290002F0D3FB0028F0D1F8E7BF
:109080002469FF1F0C69FF1F99A2001170B5064DDE
:1090900084006359002B05D0D87802F071FCFF22C0
:1090A0006359DA7070BDC0462469FF1F70B50600B1
:1090B0008CB00C00150000213022684602F068FCDC
:1090C00031001022684602F073FD1D2021000322AA
:1090D000684402F06DFD6846FFF7D8FD2D210400BD
:1090E00003222800694402F063FD20000CB070BD2B
:1090F000F0B50700160097B001931CAB1D78302225
:109100001EAB00910AA800211C7802F041FC10223D
:1091100039000AA802F04CFD1022002102A802F03A
:1091200037FC0722310002A802F042FD072202AB01
:109130009818631E9C41019902F03AFD02AB9C73A2
:109140002B005A1E934102AAD3730021102206A8B5
:1091500002F01EFC06221D9907A802F029FD1A2024
:1091600002ABC01806221F9902F022FD10220099BE
:109170000EA802F01DFD102202AB0EA908781C7883
:10918000013A6040D2B2087001330131002AF5D1B2
:109190000AA8FFF77BFD102212A904000EA802F016
:1091A0005FFD102206AB0EA908781D78013A6840D1
:1091B000D2B2087001330131002AF5D10AA8FFF7B5
:1091C00065FD044310222098E4B212A902F0F0FCDD
:1091D000200017B0F0BD70B50E0014008CB0010077
:1091E000102268461D0002F0E3FC3100082204A8AA
:1091F00002F0DEFC2100082206A802F0D9FC684635
:10920000FFF744FD04001022280008A902F0D0FC5A
:1092100020000CB070BDF8B506000D000024371911
:10922000AC4200D3F8BD02F033FC030A3B70631C70
:10923000DBB201379D4203D90234F054E4B2EEE7C9
:109240001C00EDE773B506000C000225002819D0BC
:10925000002917D0032101A8FFF7DDFF6B469A799B
:109260003F231A40013313436A463000937101A92A
:109270002200FFF71BFF051E04D10322E01C01A9F9
:1092800002F0EEFC280076BD03785807DA08C00F1C
:10929000D20080009B0710439B0F1843C0B2704759
:1092A00007230B40C908C9000B4303707047000037
:1092B00070B50400FFF7EAFE134DA4006359002BBC
:1092C00021D0186A002801D002F00AFC2B59986EB0
:1092D000002801D002F004FC2B59D86E002801D0E0
:1092E00002F0FEFB2B59186F002801D002F0F8FBAA
:1092F0002B59586F002801D002F0F2FB285902F0D8
:10930000EFFB00232B5170BD2469FF1F0E4B800023
:10931000C35870B50C00002B0FD09D68002D0CD0E9
:109320002B78201D0B706B784B70A97CFFF7B8FF72
:109330002B7E23726B69E36070BD10220021200038
:1093400002F026FBF8E7C0462469FF1F014B1860B6
:109350007047C0462069FF1F074A030080008258FB
:1093600010B5002A06D0D088984203D1012901D136
:10937000FFF79EFF10BDC0462469FF1FF0B5264EC3
:1093800095B087000B93BB590500099112200A92F2
:10939000002B31D0D888FFF7A5FB04001420002C47
:1093A0002AD0280010A9FFF7B1FFBB591E781D6A0B
:1093B000002E23D00895FDF7EFFA07000020FDF7F7
:1093C000F1FA0790A379E61D069310AD0CA9089851
:1093D00000F0E2FA0EA9280000F0D7FA0B9B0A99D8
:1093E0000493069B09980293079B039601930097A9
:1093F0000EAB0CAAFFF77CFE15B0F0BDFDF7CCFA62
:1094000006903000FDF7CEFAE31DA779079310AB65
:1094100006000893DAE7C0462469FF1F30B50C4CFC
:1094200085002A59030085B00120002A0ED01800BB
:109430006946FFF76BFF2B591A78D888054B002A2D
:1094400000D1054B6A46072100F0D9FB05B030BDBD
:109450002469FF1F8B9900119999001130B5094CAF
:109460008500295985B010226846253102F0F8FBA5
:109470002A591121044BD0886A4600F0C0FB05B080
:1094800030BDC0462469FF1F359A001130B5094C24
:109490008500295985B010226846353102F0E0FB7D
:1094A0002A591121044BD0886A4600F0A8FB05B068
:1094B00030BDC0462469FF1F739A0011F7B54D4FA8
:1094C00086001020F4590D0002F0A2FBF35920622F
:1094D000186A132200286CD0033A29009C6802F015
:1094E000BFFBF3591A780192002A58D11E6A227DD7
:1094F000317B944651400122019F114201D16746C0
:109500001740217D914339432175377B4F40BC463D
:1095100060460027800701D44F0817400121022030
:109520008F40227D82433A432275377B5740BC46A9
:1095300060460027400701D497080F400420227D91
:10954000BF0082433A432275627D002794466046FD
:10955000727B42400A4201D167460F400121627D81
:109560008A433A436275777B5740BC466046002782
:10957000800701D457080F400220627D7F0082439C
:1095800017436775767B00227E40760701D4BA08C0
:109590000A400426617D9200B1430A4362756A78ED
:1095A000002A08D06278002A05D005220533DA7730
:1095B00000221000FEBD04222979114205D1A17CB0
:1095C000114202D10533033AF1E7019A21782C7850
:1095D000002A02D10A002100140018220429E8D828
:1095E000042CE6D805206043034A05331218525C68
:1095F000DDE7C0462469FF1FF0C0001110B50A0066
:109600001121024B00F0FBFA10BDC046CF9A0011A9
:109610000B0030B587B001AD2B806B460400110004
:10962000981D082202F01CFB2A000B212000024B8F
:1096300000F0E5FA07B030BDF79A001110B50A0046
:109640001121024B00F0DBFA10BDC0464B9B00110C
:1096500013B50B0011006A4613706B460400062216
:10966000581C02F0FDFA6A4608212000014B00F068
:10967000C6FA13BD6B9B001110B50A001121024BF5
:1096800000F0BDFA10BDC046BB9B00117FB50500C0
:109690000B4BAA00D4580800002C0FD0666F237F14
:1096A000E28821780396266F0296E66E0196A46EF4
:1096B0000094FDF709FC2800FFF7FAFD7FBDC046C6
:1096C0002469FF1F10B51721FFF7E0FF10BD000050
:1096D00070B50A000D00064B0221040000F08FFA5D
:1096E000060029782000FFF7D1FF300070BDC0468A
:1096F0009B9A001170B586B000236A461370836888
:1097000004001D78681E0A2859D801A902F068FAD9
:10971000060633373B3F43474B4F5300180000F0DA
:1097200042F9062312284BD000281BD16088FFF78E
:10973000D9F90823002813D04279002A47D1264BB3
:109740001A78072312070BD5244B1A680723002A1F
:1097500006D01668002E03D0290001AAB0470300E6
:109760006A4613706B461B786088002B2AD1FFF77E
:1097700067FC06B070BD180000F06CF9D4E7180063
:1097800000F087F9D0E7180000F093F9CCE7180053
:1097900000F0ADF9C8E7180000F0C3F9C4E71800FD
:1097A00000F0F6F9C0E7180000F0F6F9BCE7180081
:1097B00000F013FAB8E7180000F013FAB4E7072333
:1097C0006A46137069466088FFF782FFD1E7052378
:1097D000012AC5D1024BB8E7B167FF1F1C69FF1F03
:1097E0002069FF1FF8B52C4F8600F35904000D00C7
:1097F000002B40D0DA8882423DD15A78062A33D1F4
:109800001A78002A2ED0012099681A6A097D01422F
:1098100006D0157B054203D007225A700120F8BDFF
:109820000220014204D0157B054201D00922F4E751
:109830000420014204D0127B024201D00B22ECE74B
:10984000164B1B68002BE9D05B68002BE6D020008C
:109850009847BB5900215B78122BDFD12000FFF71E
:1098600015FFDBE70E4BECE7112A04D1002900D0ED
:1098700032252900F2E7002D08D12000FFF732F948
:10988000002803D01023027913430371210028001C
:10989000FDF798FAC2E7C0462469FF1F1C69FF1F45
:1098A0002069FF1F70B50E4E8500AB590400002BD8
:1098B00013D01B78002B11D10A4B1B68002B04D04E
:1098C0005B68002B01D02000984773595B78122BFE
:1098D00003D100212000FFF7D9FE70BD024BECE759
:1098E0002469FF1F2069FF1F1C69FF1F094B8000AF
:1098F000C3581020002B0CD01A6A002A09D09B688C
:10990000002B06D0127A1B7E101C9A4200D9181C1C
:10991000C0B270472469FF1F70B503000D0014002A
:109920000220002A30D000292ED013700B78081D99
:1099300053704B789370FFF7A7FCE0700120022171
:109940002B7A23716B7B034063716A7B0A4013435C
:10995000042263716E7B1640334363716E7BF6089D
:10996000F600334363712B7B0340A371287B0140D6
:1099700000200B43A371297B0A401343A3712A7B68
:10998000D208D2001343A37170BD10B50A000100C4
:109990000120FFF7C1FF10BD10B50A000100022031
:1099A000FFF7BAFF10BD70B506000C000220002EB4
:1099B00030D000292ED07378201D0B70B3784B70F7
:1099C000F178FFF76DFC01223579257271794B1022
:1099D000080013409340104003438810104080005B
:1099E000C9080343C9000B436373B1794B100800E6
:1099F0001340934010400343881002409200C9086E
:109A00001343C9000B4321202373FCF773FE8542E7
:109A100001D2122070BD2220257AFCF76BFE854210
:109A2000F7D823781820042BF4D86378012BF1D8C9
:109A30000020EFE7030010B50220002909D0002B19
:109A400007D00322481C0A7019000D3202F008F9F1
:109A5000002010BD03000222080010B5002B06D024
:109A6000002904D00E32591C02F0FAF8002210002E
:109A700010BD030010B50220002909D0002B07D02B
:109A80000422481C0A7019000C3202F0E9F8002088
:109A900010BD10B5FFF7DEFF10BD03000220002946
:109AA00006D0002B04D0052200200A701B784B70D2
:109AB000704703000220002B08D0002906D05B78F5
:109AC00000200B70013B082B00D9183070470300B1
:109AD00010B50220002909D0002B07D00622481C0F
:109AE0000A7019000A3202F0BBF8002010BD10B550
:109AF000FFF7B0FF10BD02000B00022010B50029D7
:109B00000ED0002A0CD007211970118859701188C5
:109B1000090A997011180822D81C02F0A1F8002037
:109B200010BD03000A00022010B5002B0CD0002944
:109B30000AD099785878090201431180901CD91CE9
:109B4000082202F08DF8002010BD030010B502209D
:109B5000002909D0002B07D00822481C0A701900E0
:109B6000921802F07DF8002010BD02000B000220C8
:109B700010B500290BD0002A09D0092119701178DD
:109B800018185970511C062202F06AF8002010BD06
:109B900010B5FFF75FFF10BD02000B00022010B5EB
:109BA000002A09D0002907D051781970111806220F
:109BB000581C02F055F8002010BD030010B502201B
:109BC000002909D0002B07D00A22481C0A7019006E
:109BD000063202F045F8002010BD10B5FFF73AFF3D
:109BE00010BD02000B00022010B5002A06D000298B
:109BF00004D018005178FFF753FB002010BDF0B5DA
:109C000085B017001E006A460623050008009181F2
:109C10009380FEF7C0FC1324011E02900CD0380084
:109C2000B047041E05D1280001A9FEF76FFA041EF3
:109C300002D0029802F07CF82800FFF701FA200019
:109C400005B0F0BDF0B504008BB001911500002106
:109C5000102202A801F09CFE334EA700B85900283C
:109C60003CD0C388A34239D10378002B36D1427847
:109C7000062A18D102000100553235310C3006ABEE
:109C8000FFF7A9FA002829D12000FFF72FFE0200D4
:109C900006A902A801F0E4FF200002A901F010FECD
:109CA00001200BB0F0BD816E002917D00B8A112A5C
:109CB00028D19D420ED101981231093A01F0C8FD18
:109CC000012807D1BB5920009D6EFFF70FFE290028
:109CD0000200DEE732212000FFF7D8FC2000FEF76B
:109CE00001FF061E1BD0416A002918D00B8AAB4227
:109CF00015D108220198123101F0AAFD01280ED1D8
:109D0000716A0AE09D42E9D108220198123101F0FE
:109D10009FFD0128E2D1BB59996E8A7EB9E72000E8
:109D200001F036FDBCE7C0462469FF1FF0B56B4D5E
:109D300087007E5985B0337802900393002B00D0C2
:109D400087E0B368346A01937078062817D101223E
:109D50001B7D134202D0217B114218D102221342F3
:109D600002D0217B114251D10422134203D0237B24
:109D7000134200D08BE0019B5A7DEB5991E00738EC
:109D80000428F8D801F02CFF032E42678300B36E3D
:109D9000002B03D11C2001F03BFFB066EB599C6EF9
:109DA000002C1CD010220021200001F0F1FD0298AF
:109DB000FFF79CFD01002000FFF72DFA01F068FE7F
:109DC0002082200008211230FFF725FA0298FFF7C1
:109DD0008DFDA076EB592100D888FFF70FFC0822F3
:109DE000EB591CE0B36E002B05D01A00198AF088DD
:109DF0001232FFF70DFC0222019B197DEB59114233
:109E00003DD0207B10423AD0073208E0F488FCF7BE
:109E1000DBFD01002000FFF711FC0A22EB595A700C
:109E2000029B9C002A595378073B042B11D8D088F9
:109E3000FEF758FE00284ED0C3895A08D218284988
:109E4000029B0298CB542B5941180433254801F04A
:109E5000DFFD05B0F0BDFCF79FFD0300012083424C
:109E600001D100200393EB59DE88FCF79BFD039999
:109E700002003000FFF7ECFB019AEB59117D042240
:109E800011420CD0217B114209D00B22C7E7F68882
:109E9000FCF73CFD01003000FFF7EEFB6BE7019A99
:109EA000527D01210A4204D0607B084201D00C227D
:109EB000B5E702210A4204D0607B084201D00E229D
:109EC000ADE704210A4204D0627B0A4201D010228D
:109ED000A5E71222A3E7FA225200B0E72469FF1F88
:109EE0002869FF1FA3A2001110B5064B1A7804239E
:109EF000100018401A4200D00348FFF727FA00204C
:109F000010BDC046B167FF1F3446FF1F70B5040087
:109F1000FFF7D4FA051E43D12000FFF77FFA234E46
:109F2000A400A0598268937CDB0708D50321036A4B
:109F30001B790B40012B02D1017F0B430377431D9B
:109F4000D97F8B1E022B0DD8022900D00121C08899
:109F5000FCF790FF042133591A7F59700A431A778E
:109F6000280070BD01290CD102231022437000216A
:109F70000C3001F00DFD305910213530FFF74BF951
:109F8000EEE70529ECD10223D118437010220C30E2
:109F900001F066FE04233259117F0B431377EAE781
:109FA00008251828DCD1053DDAE7C0462469FF1FE3
:109FB000F0B58BB0059143887E4F9E00F459150093
:109FC0000493002C15D1012902D000200BB0F0BD64
:109FD000101D57781678FFF757F9EB683200029397
:109FE0002B7A0499019300903B002000FCF70CFFB2
:109FF000EBE7E388049A934201D00820E6E7237850
:10A00000012B00D1D4E0059B581E092800D9CFE0D0
:10A0100001F0E6FD05CE0A29CC506C859AB22900E4
:10A020000498FFF773FFD1E7200029001022453084
:10A0300001F016FEB9594B78042B02D1013B4B704D
:10A04000C3E70B000A00253335320C310498FFF7C3
:10A0500095F90498FFF702FA0522431E9841BB596F
:10A06000C0005A70B2E7200029001022553001F0DC
:10A07000F7FD049B4F4C9D00295904980A0006AB3C
:10A0800055320C31FFF77AF929591022453106A8CB
:10A0900001F0DEFB012808D10498FFF7F7F90590DD
:10A0A000002804D106222B595A7005988EE7082300
:10A0B0000593FAE763780C2B7AD1E36E002B03D17A
:10A0C0001C2001F0A5FDE066BB59D86E00286FD0BA
:10A0D0001022290001F0C4FDBB590498DC6EFFF783
:10A0E00005FC0D22A076BB595A706EE7E06E002881
:10A0F0005ED063780D2B5BD12B8808220382A91CCC
:10A10000123001F0ADFDBB599A68517D0222114217
:10A1100026D0186A407B104222D00C32E4E76378E4
:10A120000E2B45D1236F002B03D1162001F070FDBB
:10A130002067BB59186F002803D01022290001F0B6
:10A140008FFD0F22BB59CFE763780F2B30D1206FE3
:10A150000622691C103001F083FDBB599A68517DBD
:10A160000422114203D0196A497B1142D5D1002142
:10A170000498FFF78BFA28E7636F002B0DD0BB59CB
:10A18000586F0028F3D01022290001F069FD012248
:10A19000BB5952425B6F1A61E9E7142001F038FDA8
:10A1A000BB5960675B6F002BE9D126E72978DFE7B1
:10A1B00007200BE72469FF1F10B5064C207001F043
:10A1C0007FFC06212078FDF791FF0348FEF778FC1D
:10A1D00010BDC0463769FF1F5993001100200BB214
:10A1E00070B50D00834216DA264B187801F0E0FDB9
:10A1F000041E0DD00378922B0ED0A02B37D0224B0B
:10A200001878FF283AD0210001F04AFB002835D108
:10A2100080200002684070BD43780E2B0BD03E2B8F
:10A22000EDD18378052B12D0082BE8D18179808875
:10A23000FFF7D8FA08E0154B82889A42DFD183688D
:10A240001878591CFEF7C0FE002817D1D7E7104B2D
:10A250001B785B0712D50F4B1B68002B0ED09B6839
:10A26000002B0BD0C289811D80889847ECE7FFF74F
:10A2700041FAA068002801D001F05AFD200001F049
:10A280007FFCC5E73769FF1F2D46FF1F1820000020
:10A29000B167FF1F2069FF1F10B50078FFF712FAA2
:10A2A00010BD10B50078FFF7FDFA10BD0C23434335
:10A2B000084A10B59B185A68002A03D0012901D119
:10A2C000904710BD9B68002BFBD00029F9D198471F
:10A2D000F7E7C0465469FF1F01238340094A10B5C0
:10A2E000946B1C439463506B98435063D46B200071
:10A2F0009843012901D120001843D063116B0B430F
:10A30000136310BD00800040F0B500240127154BF9
:10A3100085B0DA6B144E03921A6C0192DA64019BD9
:10A32000E3403B4217D0039DE5403D400295E5B236
:10A3300002992800FFF7BAFF316A736A002908D032
:10A340003900002B01D0029979402800FFF7C4FFA3
:10A3500001E0002BF9D101340C36172CDFD105B008
:10A36000F0BDC046008000403869FF1F064B012148
:10A370005A68C2400A4204D01B68C3401800084013
:10A3800070471B6DF9E7C046008000400122064B74
:10A390008240002903D0D9680A43DA607047D9683F
:10A3A0009143D960FAE7C0460038004030B5032435
:10A3B00044430F4BE25C1B199C785D7801232D1BF5
:10A3C0000135AB40013BA340A140DB430C00122808
:10A3D00007D80849920052181168194021431160AA
:10A3E00030BD054A11680B4023431360F8E7C046AF
:10A3F00037C1001108F0004014F00040C21F70B5D2
:10A40000D4B20623092C0BD80125084C954000290D
:10A4100008D00021FFF7CAFF23682B4323600023E5
:10A42000180070BD2368AB43F8E7C0460038004011
:10A43000214BF0B51B185B78022B21D10324444338
:10A440001E4A1F4EA35C1219947801221500854004
:10A45000B76B013CE4B23D43A240B563194C1228EE
:10A4600015D89B0000290CD117495B1899680A433D
:10A470009A600123205C154A834011680B431360E6
:10A48000F0BD11495B18996891439960F1E70E4B53
:10A4900000290DD159690A435A61225C1328E8D07A
:10A4A0000123203A93400A49086803430B60E7E719
:10A4B000596991435961F0E73869FF1F37C10011AD
:10A4C000008000407CC1001100F00040A0F000407E
:10A4D000A4F00040F8B500241B4E1C4D1C4B1B5D26
:10A4E000012B1FD1194A9269E2401A420BD0012276
:10A4F000B25693402200143AD2B2022A09D8154922
:10A500004A6913434B61013402360C35172CE5D1EF
:10A51000F8BD0022B2560F499200521891680B43C1
:10A520009360F0E7022BEED1E7B23800FFF71EFF91
:10A5300001235840C1B23800FFF77AFF3800FFF717
:10A5400015FF6877DFE7C04609C100113869FF1FB2
:10A550003969FF1F00F00040012202388240054B9C
:10A56000002903D059690A435A61704759699143D8
:10A570005961FAE700380040F8B50E0001210F00DC
:10A580008740114A0400D368FD43BB43D360831E58
:10A590008B4201D8FFF7E0FF00212000FFF72EFFDC
:10A5A0000A4A0B4B5168012E05D139431B195160E2
:10A5B0005E700020F8BD2940516002221C196270B3
:10A5C0009A6915409D61F4E7003800400080004022
:10A5D0003869FF1F012210B58240074B002906D0C1
:10A5E00019680A431A600121FFF7C6FF10BD1968F8
:10A5F00091431960F7E7C046008000400C2370B516
:10A60000002543430A4A29009B181D70094B04008A
:10A610001B185D70FFF7B0FF0123A3400649280017
:10A620000A681A430A6005490A689A430A6070BDBD
:10A630005469FF1F3869FF1F34800040308000409C
:10A6400070B504000E00FF2813D003250540FFF766
:10A65000D5FF084AA3089B009B183F22ED00AA40A3
:10A66000AE40196820009143314319600121FFF782
:10A670008DFE70BD18380040F8B50C244443134BD0
:10A680000500E4186368002B03D1A3681220002B97
:10A690001AD0022201270E4B00215B195A702800A4
:10A6A0002770FFF769FF63681E1E08D0A3683E008D
:10A6B000002B04D02800FFF759FE4640F6B22800D0
:10A6C0003100FFF709FE0020F8BDC0465469FF1FA6
:10A6D0003869FF1FF7B5C420FF222B4B80001958A3
:10A6E000002491433F3A0A431A508022274F5202D6
:10A6F000274E1A60274B1D5D002D21D0A31E012B74
:10A7000003D80121E0B2FFF727FF012D18D11F4B1D
:10A710009B69E3402B4213D0E3B218000193FFF78B
:10A7200025FE01000198FFF755FFE3B2143B022B11
:10A730001DD801217156184A8D405369AB435361AE
:10A740003B7F002B0DD0E5B22800FFF795FF2800D6
:10A75000FFF70CFE7B7F0100834202D02800FFF749
:10A76000A5FD01340C370236172CC3D1F7BD0121EA
:10A7700000237156F3568D40074A9B009B189A6838
:10A78000AA439A60DCE7C04600E100E03869FF1F99
:10A7900009C100113969FF1F00F0004070B50E00BB
:10A7A00015000400FFF72AFF0C236343094A200029
:10A7B0009B189D605E60FFF75FFFF021064B074A24
:10A7C0008900051E5A5002D02000FFF717FF28000D
:10A7D00070BDC0465469FF1F0000FF1F09A3001190
:10A7E00070B5134D07202C78002C1FD19822210022
:10A7F0005200280001F07CF90123C420FF222B70B5
:10A800000C4B80001C635C630B4B1C605C600B4B4F
:10A81000195891433F3A0A431A50802252021A6053
:10A820000D20074A074901F063F8200070BDC046BB
:10A830003869FF1F00800040A0F0004000E100E008
:10A84000D5A60011D5A40011030010B50620072BD2
:10A8500009D8054A137001F0D3FAD7210020034B21
:10A86000034A89005A5010BD5C46FF1F0000FF1FBD
:10A87000151BFF1F70B51D0002240C2910D8094AB2
:10A88000CA40D2070CD5FBF741FF041E08D1059A38
:10A8900004992800FBF756FFFCF7C4FDFFF724FBE3
:10A8A000200070BD1210000030B50D7802232C007E
:10A8B0009C43184201D02B431C0008252300AB43C6
:10A8C000284201D02B00234320241D00A543204211
:10A8D00001D01C4325002A230D70184204D01178A2
:10A8E0001E3B0B43137030BD0028FCD10C211378A4
:10A8F0008B43F7E7F8B51D0006AB1B88140007AAC9
:10A900000E000B201778002B27D10A78022A49D194
:10A910004A68507811780002244A084380180428B5
:10A9200040D801F05DF903121D1B2300F06801F00F
:10A9300087F9021CC0B2B84200D93A1CD2B220003A
:10A94000F1682A8001F08CF906E00222F3681B8886
:10A950002A8023701B0A63700020F8BD0622EEE7F0
:10A9600001232B80F3681B782370F5E7F368002B35
:10A9700016D008222A801A8822701A88120A627059
:10A980005A88A2705A88120AE2709A8822719A88AC
:10A99000120A6271DA88A271DB881B0AE371DBE7B5
:10A9A0002B80D9E701202B80D7E7C04600D6FFFFD8
:10A9B000F7B516000A781D0008AB1F880C000123AC
:10A9C000022A18D14A685078117800022B4A0843AD
:10A9D000801803280FD801F003F902254439E068F4
:10A9E00001F02EF9C0B20723B84204D37B190193BA
:10A9F000152B02DD0D231800FEBDE0682A00310092
:10AA0000C01901F02DF96B4600209B88E268D054F4
:10AA10001B4B1B68834203D01B68834200D09847BE
:10AA20000023E8E70B23002FE5D1022DE2D1737854
:10AA300032781B021343E2681380114B1B68002B12
:10AA4000EED01B68002BEBD00120E8E70B23002F92
:10AA5000D1D1062DCED12A003100E06801F000F9F5
:10AA6000DEE70B23002FC6D1012DC3D13278753319
:10AA7000012AC0D8E3681A70D2E7C04600D6FFFFAB
:10AA8000446BFF1F70B50C001500072837D801F084
:10AA9000A7F8041436361B36242E182015290BD897
:10AAA000184E16220021300000F072FF220029000B
:10AAB000300001F0D5F8002070BD18200229FBD12C
:10AAC0001288114B1A80F6E718200829F4D10A00E1
:10AAD0000E48290000F024FFEDE718200129EBD1F2
:10AAE0000B4B10780B49DA69FFF7DEFEE3E718201D
:10AAF0000129E1D1064B10780749DA6BF4E702200F
:10AB0000DAE7C0462C6BFF1FDA46FF1FD046FF1F57
:10AB10006046FF1F8846FF1FA846FF1F030010B5B1
:10AB20000020DB0704D50721024A034800F08CF817
:10AB300010BDC04694C100116046FF1F054A0300C6
:10AB40001068002803D082889A4201D1806870473B
:10AB50000068F6E7486DFF1F0A88030008009A4264
:10AB600004D08A8804309A4200D000207047000048
:10AB7000F8B5F82200230D4F0D4E796805004243C9
:10AB80003370994200D07B600A4C0021200000F015
:10AB9000FFFE00231A007C60AB4202D1002033701C
:10ABA000F8BD01332280DBB2F834F5E7486EFF1FB1
:10ABB000446EFF1F4C6DFF1F73B56B46019006007E
:10ABC000684615001980FCF75FFF041E11D1002DA7
:10ABD0000FD07689002E11D00C2001F019F8002832
:10ABE0000ED0084A0460136886808560002B02D16D
:10ABF0001060200076BD1A001B68F7E70224F8E712
:10AC00001324F6E7486DFF1F012100220A4B10B5FF
:10AC100049420A4C198099809A719A70084B2070A9
:10AC2000012019805A60FFF7A3FF2078FCF78AFF04
:10AC30000448FDF745FF10BD4C6BFF1F506EFF1F12
:10AC4000486EFF1FF5AC0011022310B5002802D09A
:10AC5000FFF7B2FF0300180010BD0000030010B59D
:10AC60000020DB0704D50421024A0348FFF7A4FFB4
:10AC700010BDC046A8C10011E046FF1FF0B50E266A
:10AC800087B003930CAB1F8802ABF61805000800D1
:10AC900031000292FDF77AF804000120002C0FD059
:10ACA0003088FFF74BFF03000E20002B08D05E68B2
:10ACB000002E05D021002800039B029A0097B04780
:10ACC00007B0F0BD0A4B10B5984207D1012200230E
:10ACD00052420A808B708A808B7110BDFFF73CFF57
:10ACE0000028FAD001235B42038000238370F4E73D
:10ACF000FFFF0000F8B5050001290AD1134E00241A
:10AD00003388F827AB4219D028001149FFF7DAFF42
:10AD100006E0022904D10139FDF750FF0028EDD0EB
:10AD2000F8BD3B0063437268D018D35A002B09D09A
:10AD30003A00002100F02CFE0134E4B2054B1B78F0
:10AD4000A342EED801235B423380DDE7486EFF1F4C
:10AD50004C6BFF1F446EFF1F10B5FFF7FDFE030095
:10AD60000020834200D0987810BD0000F0B589B073
:10AD70001C000EAB80CB03901E8810AB1B78049296
:10AD800002930B7A0D00DB0616D42B780593022B69
:10AD900024D00498FFF7D2FE002812D003689C4606
:10ADA000002B0ED0029B2200019329003B00644639
:10ADB00003980096A04705E00498FFF7BFFE00281F
:10ADC00002D10E2009B0F0BD8368002BF9D00A2211
:10ADD0002900039898470028D7D0F3E76B68587884
:10ADE0001A786B4B000210439842D2D8043B984229
:10ADF00010D2684B984242D015D8674BC018012832
:10AE0000C7D80B20002EDDD1EB681A7859683A803C
:10AE1000200028E0614BC018032800D979E000F039
:10AE2000DFFE846A789E5E4B9842B2D10B20002EE2
:10AE3000C8D101233B80EB6831001B7823706889FF
:10AE4000013080B2FCF7A2FF3A88031E0ED00178D1
:10AE500002328A183A80428962704289120AA270CC
:10AE600059680278E01C00F0FBFE06E004323A80EC
:10AE700031000422601C00F08BFD0020A2E70B20B3
:10AE8000002E9FD1EB6807A91E8804233B80330A5C
:10AE9000300026706370FCF779FF051E28D004ABE4
:10AEA0009A890E2304A95B183E49C668FCF7E2FFA5
:10AEB00000280BD12B783C486A680599FBF798FB72
:10AEC000002803D1012304AA5B42D3813278022AED
:10AED00006D17168201D00F0C3FE3B8802333B8021
:10AEE0000E2304AA9B181B88A3701B0AE370C4E7F7
:10AEF00004ABDE81F4E70B20002E00D062E7E968A6
:10AF00000398FFF729FF02233B802070000A60703E
:10AF1000B3E70B20002E00D054E70222EB681B8819
:10AF20003A8023701B0A6370A7E7E86800F088FE88
:10AF3000C2B203000720B24200D243E70DD002990B
:10AF4000DBB27118994202DB921BD3B20293029BCF
:10AF5000E9681A003B8089195AE70023F6E70B20BD
:10AF6000002E00D02EE70722EB683A801A78227074
:10AF70005A7862705A88A2705A88120AE2701A7956
:10AF80002271DA886271DB881B0AA37175E7C046FB
:10AF9000042900000228000000D8FFFFFFD6FFFFB1
:10AFA00003280000FFFF0000D8C00011F0B58DB0ED
:10AFB0006B460020089120229B5E83423DDAA64B1F
:10AFC000187800F0F5FE071E32D00378B02B2CD194
:10AFD0000079023816281FD800F0C2FC17001E00A6
:10AFE0001E001E0031001E0096001E001D011E00E6
:10AFF00052011E0073011E00CD011E0050021E00F2
:10B000001E001E008E021E00E302944B94491B8812
:10B0100078880B80FBF72CF83800FCF7ADFF914BDC
:10B020001B68002B01D038009847380000F0A8FDBD
:10B030008020089B0002434018000DB0F0BDF622AE
:10B040000021874800F0A4FC0BAA3B7B7989388952
:10B0500000923A000D32FCF7B1FD0400804B1B78E2
:10B06000002C3FD146E0804B788805937F4B410010
:10B07000CB5A0BAE073BDBB232880293002301931D
:10B080007B4B210006930093059BFFF76FFE744DE9
:10B09000002810D1069B3A8A1B889A420BD13800AF
:10B0A0000599123000F0D4FB002804D02B78628977
:10B0B0009B00EB185A80162306A81B183288200024
:10B0C0007989FCF7D7FE2B7804009A00AA185188DA
:10B0D0000029C3D00133DBB22B70002807D006A9AA
:10B0E000C98A9180634A12889A42BCD802E0012141
:10B0F00049429180002B04D059497888FAF7ECFF37
:10B100008AE73E890A2479E000253E89574B069359
:10B110007B88069A5B009B5A033B9D4202DB002D15
:10B12000F0D05BE0162206A812183B7B79890092CA
:10B130003A0030000D32FCF741FD0590002858D050
:10B140004689017A7888FCF703FD041E44D1464BFA
:10B1500078880793069B4100C95A454B0439C9B208
:10B1600006AAD28A06930291019400930599079B3F
:10B17000FFF7FCFD041E2FD1069B39491A88931C4A
:10B18000002D26D14B807988384B4900CB5A511974
:10B19000033B8B4220DD059B31485B8941190B71D4
:10B1A000A91C0135C9B2EDB2059145191B0A2B71D5
:10B1B000059B2D490433181800F052FD2C4B059ABD
:10B1C0001B88D318DDB22C4B9E4205D00136B6B297
:10B1D0009CE749889942D6D0002D0CD0204C2800FD
:10B1E000618800F02DFE207021007888FAF784FF36
:10B1F00012E7059CF0E7002C00D183E77B78142B45
:10B2000000D109E716493B794E800B700C717888A4
:10B21000FAF724FF00E7162406ABE418210038896A
:10B22000FCF7B4FD011E00D1B7E1788822880F4CED
:10B2300045002C5B0A4D013CE4B2029400240F4B04
:10B2400001940095FFF792FD041E00D014E129003F
:10B250007888FAF761FFDFE6506EFF1FCC45FF1FCD
:10B26000546BFF1F486BFF1F4E6CFF1F8467FF1F4F
:10B27000446DFF1FCA45FF1FFFFF0000566BFF1FF5
:10B28000162406ABE41821003889FCF77FFD011E67
:10B2900000D182E178882288AE4C45002C5BAE4D0F
:10B2A000013CE4B202947C89AC4B01940095FFF719
:10B2B0005DFD041E00D0DFE029007888FAF736FF34
:10B2C000AAE60025A44B1D803B00FE331B78A24A52
:10B2D00078880792AB4208D99E4B1288069306994C
:10B2E00043005B5A013B9A4203DB0799FAF728FFB8
:10B2F00092E616246B00FB18059306ABE418059B39
:10B3000021001889FCF742FD011E03D1059B012491
:10B310001E8973E77888924B2288069C0993430024
:10B320001B5B904E013BDBB202930023009601931E
:10B33000099BFFF71BFD041E02D0059B1E895DE7DC
:10B340007B88069A5B009B5A079A108832881218ED
:10B35000934202DC1B1A013B33807F4C023032885F
:10B360000999001900F07CFC2388328801359B186C
:10B370002380EDB2A8E70BAA3B7B7989388900923C
:10B380003A000D32FCF71AFC00250590059B002BB6
:10B3900004D10A24002D00D16EE060E0059B78887E
:10B3A000197AFCF7D5FB0100041E63D1694C6C4B84
:10B3B000788806940993069B4400E45A694B063C3E
:10B3C000E4B20BAE32880793029401910093059981
:10B3D000099BFFF7CBFC041E4CD1079B5E491B88E1
:10B3E0001A1D002D30D14A80059B5B4C5A89631988
:10B3F0001A716B1C9BB2E318120A1A71162306A865
:10B4000032881B1879890598FCF734FDFF21AA1CA6
:10B410002E1D03350B00059092B2B6B2ADB20028D6
:10B4200003D006ABDB8AD9B21B0AA21865191171C9
:10B430002B714C4D301D2A884949201800F010FC12
:10B440002B88F618B5B2A1E74988914207D17A88CE
:10B4500006995200525AEB18053A9A42C4DC3E4C07
:10B460002800618800F054FB207021007888FAF7EA
:10B4700071FED1E5002DF2D13E89BFE6162606AB5E
:10B48000F61831003889FCF781FC3D000400FF35D7
:10B4900000282DD0037A9B060CD400227B893989A1
:10B4A000788800923A000C32FFF7E8FB041E10D0B7
:10B4B0003E8915E03088FFF741FB00281AD08368E9
:10B4C000002B17D02100122278889847041EE4D060
:10B4D000EEE7AB78002B02D17888FAF74BFE002616
:10B4E000AB78002B00D097E5002C00D194E585E6E1
:10B4F0000124DDE70E24DBE7162506ABED18290055
:10B500003889FCF743FC041E47D0037A9B0611D40C
:10B51000154A7B881188994203D01448814207D18B
:10B520001380134BF8261D780023D9B2A94221D3EA
:10B530000924A1E72888FFF701FB00282FD08368A2
:10B54000002B2CD02100122278889847041EDFD0CF
:10B5500092E7C0468467FF1F546BFF1F566BFF1FA7
:10B560004E6CFF1F446DFF1F486EFF1FFFFF000062
:10B57000446EFF1F31005943546801336018615A0B
:10B580000029D2D13C0008342100F82200F068FBE9
:10B5900021007888FAF7F6FD3EE501246CE70E24D9
:10B5A0006AE71D4B1A887B889A4231D07888FAF76F
:10B5B000F3FD31E5F823059851684343CD18C95A86
:10B5C00000291FD03B7A012B0BD16C88AB8878887F
:10B5D000AA1D0094FFF752FB041E02D000233B7209
:10B5E0002E88F8220021280000F0D2F900232B80B9
:10B5F000059B0133DBB20593084B05991B78064A7E
:10B600008B42D7D801235B421380002CCED0F5E5C6
:10B61000002634000596EFE7486EFF1F446EFF1FBB
:10B6200070B504000E001500FFF796FA031E08D14E
:10B6300031000548FFF790FA03001120002B02D0DB
:10B640001C8000209D7070BDFFFF0000F8B50B4FFF
:10B6500006003B780D001400FF2B0ED00A2000F0EE
:10B66000B7F9011E09D0B12303800023468003717E
:10B67000C5800481387800F013F9F8BD2147FF1F19
:10B68000F7B50F0008A90600088809A90B24098846
:10B69000002821D10234022B1ED1557813782D02B7
:10B6A0001D432B008B4301937334002B14D1FB6893
:10B6B000300019000093FFF74FFB019C85420BD02F
:10B6C0002A0030000099FFF7ABFF041E04D12A00C6
:10B6D00030007989FFF7BAFF2000FEBDF0B50E7883
:10B6E00085B003900AA805880120022E0DD14C6870
:10B6F0002778647824023C43054FBC4205D1039867
:10B70000DBB201960095FFF7BBFF05B0F0BDC04668
:10B710000229000010B504000C4800F0E1F80C48C4
:10B72000A16B00F0DDF80B48E16B00F0D9F80A4896
:10B73000216C00F0D5F8094B0948196800F0D0F8E1
:10B74000084B1B68002B00D09847FEE78ABF00110A
:10B75000A0BF0011AFBF0011BEBF001104ED00E09B
:10B76000CDBF0011546EFF1F002307B501A8019340
:10B77000FFF7D0FF044A0548002110B5121A00F067
:10B7800007F9F8F71DF9FEE7586EFF1F2447FF1F62
:10B7900001B40248844601BC604700BF091B000099
:10B7A00001B40248844601BC604700BF8534FF1FD6
:10B7B00001B40248844601BC604700BF4532FF1F08
:10B7C00001B40248844601BC604700BF2526000042
:10B7D00001B40248844601BC604700BF9D32FF1F90
:10B7E00001B40248844601BC604700BFE117000075
:10B7F00001B40248844601BC604700BFA54F010068
:10B8000001B40248844601BC604700BF056A0000DD
:10B8100001B40248844601BC604700BF350E0000F9
:10B8200001B40248844601BC604700BF5147010093
:10B8300001B40248844601BC604700BF4D1F0000B0
:10B8400001B40248844601BC604700BF554901006D
:10B8500001B40248844601BC604700BFCD4C0100E2
:10B8600001B40248844601BC604700BF013BFF1F92
:10B8700001B40248844601BC604700BFC534FF1FC5
:10B8800001B40248844601BC604700BF3555000042
:10B8900001B40248844601BC604700BF6DBC000093
:10B8A00001B40248844601BC604700BF594F010003
:10B8B00001B40248844601BC604700BF8938FF1FBD
:10B8C00001B40248844601BC604700BF311B000040
:10B8D00001B40248844601BC604700BFC56D010049
:10B8E00001B40248844601BC604700BFE53A01004C
:10B8F00001B40248844601BC604700BFE532FF1F27
:10B9000001B40248844601BC604700BFED4A010013
:10B9100001B40248844601BC604700BF01890000B1
:10B9200001B40248844601BC604700BF810E00009C
:10B9300001B40248844601BC604700BFC9A90000A9
:10B9400001B40248844601BC604700BFB14E00000C
:10B9500001B40248844601BC604700BF153BFF1F8D
:10B9600001B40248844601BC604700BF053EFF1F8A
:10B9700001B40248844601BC604700BF8D3BFF1FF5
:10B9800001B40248844601BC604700BF1147010072
:10B9900001B40248844601BC604700BF154D010058
:10B9A00001B40248844601BC604700BF3D18000056
:10B9B00001B40248844601BC604700BF6D30FF1FE0
:10B9C00001B40248844601BC604700BF055E000028
:10B9D00001B40248844601BC604700BF1D4D010010
:10B9E00001B40248844601BC604700BFB352010065
:10B9F00001B40248844601BC604700BF2136FF1FE6
:10BA000001B40248844601BC604700BF8B5201006C
:10BA100001B40248844601BC604700BFA94601004A
:10BA200001B40248844601BC604700BF21460100C2
:10BA300001B40248844601BC604700BF5938FF1F6B
:10BA400001B40248844601BC604700BF156B010089
:10BA500001B40248844601BC604700BFE5480000CD
:10BA600001B40248844601BC604700BF01240000C5
:10BA700001B40248844601BC604700BFE9280000C9
:10BA800001B40248844601BC604700BF595201001E
:10BA900001B40248844601BC604700BF295101003F
:10BAA00001B40248844601BC604700BF0D5201004A
:10BAB00001B40248844601BC604700BF5D32FF1FED
:10BAC00001B40248844601BC604700BFC92600009B
:10BAD00001B40248844601BC604700BF5522000003
:10BAE00001B40248844601BC604700BF014C01001C
:10BAF00001B40248844601BC604700BFB70E000095
:10BB000001B40248844601BC604700BFADAE0000EE
:10BB100001B40248844601BC604700BF090E000022
:10BB200001B40248844601BC604700BFC51D000047
:10BB300001B40248844601BC604700BFC94A010005
:10BB400001B40248844601BC604700BF090E0000F2
:10BB500001B40248844601BC604700BFC521000013
:10BB600001B40248844601BC604700BF9DA90000A3
:10BB700001B40248844601BC604700BF7D18FF1F26
:10BB800001B40248844601BC604700BF434D010038
:10BB900001B40248844601BC604700BFF94C010073
:10BBA00001B40248844601BC604700BF2535FF1F31
:10BBB00001B40248844601BC604700BF4551010002
:10BBC00001B40248844601BC604700BF691F000001
:10BBD00001B40248844601BC604700BF65710100A2
:10BBE00001B40248844601BC604700BFF13DFF1F1D
:10BBF00001B40248844601BC604700BFDD3DFF1F21
:10BC000001B40248844601BC604700BF393CFF1FB5
:10BC100001B40248844601BC604700BF3D4B0100AF
:10BC200001B40248844601BC604700BF0D3AFF1FC3
:10BC300001B40248844601BC604700BF291C0000D3
:10BC400001B40248844601BC604700BFDD520100D8
:10BC500001B40248844601BC604700BF4550000063
:10BC600001B40248844601BC604700BFE94C0100B2
:10BC700001B40248844601BC604700BF4D3BFF1F32
:10BC800001B40248844601BC604700BF85520100F0
:10BC900001B40248844601BC604700BF8D12000019
:10BCA00001B40248844601BC604700BF5D17000034
:10BCB00001B40248844601BC604700BFB54C010096
:10BCC00001B40248844601BC604700BFB930FF1F81
:10BCD00001B40248844601BC604700BF5939FF1FC8
:10BCE00001B40248844601BC604700BFC53F000064
:10BCF00001B40248844601BC604700BF456B0100A7
:10BD000001B40248844601BC604700BFE13CFF1F0C
:10BD100001B40248844601BC604700BF21240000F2
:10BD200001B40248844601BC604700BF6538FF1F6C
:10BD300001B40248844601BC604700BFD9490100F4
:10BD400001B40248844601BC604700BF5125000091
:10BD500001B40248844601BC604700BF851F000053
:10BD600001B40248844601BC604700BF5118FF1F60
:10BD700001B40248844601BC604700BFCD3BFF1FB1
:10BD800001B40248844601BC604700BF1D4B01005E
:10BD900001B40248844601BC604700BF75A9000099
:10BDA00001B40248844601BC604700BFF30E0000A6
:10BDB00001B40248844601BC604700BFF54E010053
:10BDC00001B40248844601BC604700BF79180000F6
:10BDD00001B40248844601BC604700BF017F0000F7
:10BDE00001B40248844601BC604700BFEDA50000D5
:10BDF00001B40248844601BC604700BFDD66010013
:10BE000001B40248844601BC604700BF151BFF1FF8
:10BE100001B40248844601BC604700BFD91B000042
:10BE200001B40248844601BC604700BFC95C010000
:10BE300001B40248844601BC604700BFB53CFF1F07
:10BE400001B40248844601BC604700BF350E0000C3
:10BE500000030102020303030403050006020700B6
:10BE6000080209030A030B030C000D000E030F0365
:10BE7000100311031203130314031502160200002A
:10BE80009D3D0011D13D00110000000002000000A6
:10BE900096BE0011192A0F180A000000F15900007F
:10BEA000FD24000041460100C9810011DDA10011FF
:10BEB00031760011CD7F0011A5540011ADAF0011F6
:10BEC0000D510011953F0011C54000110000000008
:10BED0001616000002000000E0BE0011F4FFF3FFA0
:10BEE000D2FC00000542001100000000000000002C
:10BEF000547579610042312E33003030313700679C
:10BF000069746875622E636F6D2F70767678005451
:10BF1000484231000200000028BF0011292A282AC7
:10BF2000272A262A252A242A0A180000E2040000CB
:10BF30007102000078EC000074400000102700003F
:10BF400060F0000006640000204E000000000000C9
:10BF5000050000001F501D00023CB4000001170046
:10BF600013000000A102000030313233343536377F
:10BF70003839414243444546005048592B363258DF
:10BF800058504C555330353034005B486172642052
:10BF90006661756C742068616E646C65725D0A0020
:10BFA0004C522020203D203078253038780A00502F
:10BFB000432020203D203078253038780A00505327
:10BFC0005220203D203078253038780A00494353EC
:10BFD00052203D203078253038780A00A9580011C9
:10BFE000FD5800110000000002000000F4BF001125
:10BFF0006F2A6E2A1A18EAD8BC80F0FC6000000094
:10C000000000000000005F066B2F363D7D077F3F7C
:10C01000777C596E7971000001A0000000000000DB
:10C020006410B71DC8206E3BAC30D9269041DC7639
:10C03000F4516B6B5861B24D3C7105502083B8EDE3
:10C0400044930FF0E8A3D6D68CB361CBB0C2649B07
:10C05000D4D2D38678E20AA01CF2BDBDFB349B5F2C
:10C06000800000800010000000000000336200111A
:10C07000BD78001157620011C57C0011DB62001110
:10C080009B7C001151630011717C0011A3630011AE
:10C09000397E00110B640011397E00113D640011DE
:10C0A000F37D001151630011297C0011C963001157
:10C0B000D17D00110000000000000000AF640011FD
:10C0C000D17D001111650011D5780011052A042ACF
:10C0D000012A002A02290328012800280118001833
:10C0E00000000000000000000000000000000087C9
:10C0F0000101020102010102010203030401030123
:10C10000010101010303020103000D000E001000F4
:10C11000110013001401070108010A010B011C01A1
:10C120001D02040205020702080219021A021C027B
:10C130001D030103020317000201000504000807A4
:10C14000000B0A001716001D1C0102010105040165
:10C150000E0D011110011413011716011A19020214
:10C1600001020B0A020E0D0211100214130217161F
:10C17000030504030807030B0A030E0D0001020365
:10C1800007090A0B0E0F101112141718191A1B1F8A
:10C1900020212200F5A80011B1A900110000000023
:10C1A00002000000DEC0001100000000DDB600113A
:0CC1B0000000000002000000DCC00011D4
:020000041FFFDC
:1000000000000000F93E00119CBE001198BE0011D6
:100010003064FF1F0000000000000000000000002E
:1000200000000000000000000000000000000000D0
:1000300000000000000000000000000000000000C0
:1000400000000000000000000000000000000000B0
:1000500000000000000000000000000000000000A0
:100060000000000000000000000000000000000090
:100070000000000000000000000000000000000080
:100080000000000000000000000000000000000070
:100090000000000000000000000000000000000060
:1000A0000000000000000000000000000000000050
:1000B0000000000000000000000000000000000040
:1000C0000000000000000000000000000000000030
:1000D0000000000000000000000000000000000020
:1000E0000000000000000000000000000000000010
:1000F0000000000000000000000000000000000000
:1001000000000000000000000000000000000000EF
:1001100000000000000000000000000000000000DF
:1001200000000000000000000000000000000000CF
:1001300000000000000000000000000000000000BF
:1001400000000000000000000000000000000000AF
:10015000000000000000000000000000000000009F
:10016000000000000000000000000000000000008F
:10017000000000000000000000000000000000007F
:10018000000000000000000000000000000000006F
:10019000E934FF1F3133FF1FC1660100000000007A
:1001A000000000000000000000000000000000004F
:1001B000000000000000000000000000000000003F
:1001C000000000000000000000000000000000002F
:1001D000000000000000000000000000000000001F
:1001E000000000000000000000000000000000000F
:1001F00000000000000000000000000000000000FF
:1002000000000000000000000000000000000000EE
:1002100000000000000000000000000000000000DE
:1002200000000000000000000000000000000000CE
:1002300000000000000000000000000000000000BE
:1002400000000000000000000000000000000000AE
:10025000000000000000000000000000000000009E
:10026000000000000000000000000000000000008E
:10027000000000000000000000000000000000007E
:10028000000000000000000000000000000000006E
:10029000000000000000000000000000000000005E
:1002A000000000000000000000000000000000004E
:1002B000000000000000000000000000000000003E
:1002C000000000000000000000000000000000002E
:1002D000000000000000000000000000000000001E
:1002E000000000000000000000000000000000000E
:1002F00000000000000000000000000000000000FE
:1003000000000000000000000000000000000000ED
:1003100000000000000000000000000000000000DD
:1003200000000000000000000000000000000000CD
:1003300000000000000000000000000000000000BD
:1003400000000000000000000000000000000000AD
:10035000000000000000000000000000000000009D
:10036000000000000000000000000000000000008D
:1003700069B700110000000000000000000000004C
:10038000000000000000000000000000000000006D
:10039000000000000000000000000000000000005D
:1003A000000000000000000000000000951AFF1F80
:1003B000000000000000000000000000000000003D
:1003C000000000000000000000000000000000002D
:1003D000000000000000000000000000000000001D
:1003E000000000000000000000000000000000000D
:1003F00000000000000000000000000000000000FD
:081838006072FF1F4118FF1F41
:10184000024981F3088802F0EFFB00006072FF1F7D
:1018500010B502F079FD072804D0122808D002281C
:1018600008D010BD044A0420136B01331363F8E75A
:101870000220F6E71420F4E72C68FF1FF8B50700F4
:101880000C0026002500503630785135002804D150
:101890000300287058342370F8BD2978CA00481E08
:1018A0008141A3183800A25C5B68C9B2FFF7D0FF82
:1018B00000280DD12B78DA00A218013350602B706C
:1018C0003378044A013B3370136A01331362D8E75B
:1018D0000123DFE72C68FF1F5C234343074910B552
:1018E000C9180B0058331B78012B05D1FFF7C6FF31
:1018F000034A936A0133936210BDC0466068FF1FBC
:101900002C68FF1F10B502F0DFFB064A012113000F
:1019100010CB4942D967044B136002F04DFB200005
:1019200010BDC04600E100E01000100010B504003A
:1019300002F0CAFB024B1C6002F03EFB10BDC04629
:1019400000E100E010B5040002F0BEFB4021094AAE
:10195000200013688B43136002F0FEFB01F0A6FD2C
:101960000022054B01201A60044B04321A6002F079
:101970009BFBFEE71CF00040C4F00040C0F00040BC
:10198000431E5A425341A022F0B5D2015B4213409C
:10199000154D164A40019B182A18127E8BB00191F2
:1019A000002A1BD01A000832D46F0022E6B206AF1C
:1019B000E4B294420EDC2818C369002B08D00199C8
:1019C00002AA117106AA049202AA167303A89847E4
:1019D0000BB0F0BD1978B9540132EAE71A7D1A78D4
:1019E00006AB01261A70E6E7EC6AFF1F00400040D4
:1019F000F0B5254B04004001C25C85B0002A2BD015
:101A00001A18117E002927D0917E002924D011793F
:101A1000022921D11689D788D168F51BADB22A1CBD
:101A2000102D00D9102292B2BE4217D118180123EE
:101A300003710023C269C38003819A4206D06846BD
:101A4000032103730171029301A890470820002C21
:101A500000D0192001F022FC05B0F0BD013C654228
:101A60006C41A0256442ED012C40084D1B186419FF
:101A7000074D0633013A92B2AA42EDD01888461CAF
:101A80001E80085C2070F5E7EC6AFF1F00400040F4
:101A9000FFFF00000F220E4B10B59868104002386F
:101AA0000A280BD802F0A4F90D0A0B0A0A110A0A37
:101AB0000A0A060002210020FFF762FF10BD012183
:101AC000F9E70020FFF794FFF8E7DB6FF6E7C04681
:101AD000004000400F220E4B10B5986810400238AD
:101AE0000A280BD802F084F90E0A0B0A0A120A0A15
:101AF0000A0A060002210120FFF742FF10BD012162
:101B00000800F9E70120FFF773FFF7E7DB6FF5E760
:101B10000090004013B5334C2378072B3DD8324B4F
:101B20001A78324B002A39D18022196852020A43AE
:101B30001A60252002F00AF820232D4A11680B4371
:101B4000802113606B460422C905086807331042E0
:101B500028D080210422C905C86810422ED08021D7
:101B60002020C905CA688243CA6014221A701A78F4
:101B7000002A2FD18021C905C86820320243CA60DB
:101B800014221A701A78002A28D11A4B1A7D22784A
:101B90005A601D221A705932DA6013BD1A6816494C
:101BA0000A40C5E7086802430A6014221A701A78CE
:101BB000002ACED01A78013AD2B2F7E7C8680243B9
:101BC000CA6014221A7019784A1ED2B21A700029FB
:101BD000F9D1C4E71A78013AD2B2C7E71A78013AC4
:101BE000D2B2CEE75C46FF1F2447FF1F3CF0004007
:101BF0005446FF1F00200040FFFFFEFF564B70B50C
:101C00001B68012B03D1554A936D0133936502F094
:101C100093FB534B534A1860534B544C1A600123A7
:101C2000534A1360534A13602378002B06D00622D0
:101C30005149524802F030F900232370504A514B69
:101C400010681B78C1B2002B0ED14F4CC0B2237864
:101C50005BB2002B4FDB237824785BB264B21B04A9
:101C600024021B191B1813600B1C50294ED950233A
:101C7000464A47491078DBB2FF2202284BD1086858
:101C8000444C454D267890432A78964254D9227880
:101C900024782E78023B5D10A31B6B435201D31AAC
:101CA00010335B111843086002F0CEF8031F012BBC
:101CB00045D83A4B1B78002B06D0394B1B78002BAC
:101CC00002D0002002F0D8F9A122364B9200997878
:101CD000354B4A431B689B18832292009B181B7844
:101CE000033B012B03D8AF20400002F075FA01221C
:101CF0002E4BDA8270BD237824785BB264B2FF3356
:101D0000FF341B0424021B190138ABE7CAB2022AB4
:101D1000AED20223ACE70868254C264D26789043C6
:101D20002A78964208D9227824782D78023B5B10D5
:101D3000641B63435201B2E72378DBB2B2E70228A7
:101D4000D5D11D4B1B78013B022B03D91B4B1B78B4
:101D5000022BCCD16C20C8E79809FF1FFC0FFF1F96
:101D60006467FF1FFF3F0000141003406867FF1FF8
:101D70000C10034000100340D50BFF1F7211FF1F12
:101D8000B40003408C09FF1F680AFF1F490AFF1FA8
:101D900094000340460AFF1F470AFF1FF908FF1F70
:101DA0002209FF1F300DFF1F3409FF1FBC0BFF1F4F
:101DB000440AFF1F450AFF1F1C09FF1F2309FF1FBD
:101DC00010B502F039FA0022014B1A8010BDC0464E
:101DD0006067FF1F10B502F087F9A121054A89004D
:101DE0009478054A61431268044B5218528C1A8049
:101DF00010BDC046300DFF1F3409FF1F6067FF1F75
:101E000010B50D4B0D4A9978A1239B004B431268E6
:101E1000D218531DD97F0A4B1B88994209D2441C02
:101E200007D0C82805D0D2695B1A5A43054B5343E3
:101E3000C01802F0C1F910BD300DFF1F3409FF1F9B
:101E40006067FF1F7102000070B5244D2B68002BE6
:101E500028D002F071F92B68D8402B680400002BC1
:101E600027D002F021FA2B68D8401D4B1D4A9978E3
:101E7000A1239B004B431268D118D25C91239B0095
:101E8000002A20D0CA580132CA50174B17491B6884
:101E90000868834214D3D23B181A012A1AD0144B73
:101EA000186070BD02F048F9124B196802F03CF955
:101EB000D3E702F0F9F90F4B196802F035F9D4E7CE
:101EC0000D495B18E8E7CA500C4B1B68DB68E41847
:101ED000201AE4E7F530FF30E1E7C0461C08FF1F99
:101EE000300DFF1F3409FF1F9C09FF1F6467FF1F90
:101EF000A009FF1F1808FF1F2DFF3F006C67FF1F81
:101F000070B504000D00282916D10300A433C2883F
:101F10001B889B1A0B4A9BB293420DD906006A3666
:101F200005223100653002F06FF9002804D131003C
:101F3000200002F0F1F870BD2900200002F0E4F862
:101F4000F9E7C046FE7F0000F8B50400012002F06A
:101F50002BF902F0C1F9174A17491060174D030019
:101F6000886A174E28607568AC46164D2F680025A4
:101F7000BC4501D275687D1B134E00193560C862DF
:101F8000A4204C6A40032043486210490978002984
:101F900005D00F490978022902D10F3B1360F8BD23
:101FA000012901D1083BF9E7032901D1053BF5E7F8
:101FB000033BF3E7E408FF1F00F00040340AFF1F73
:101FC00028100040180AFF1F1C0AFF1F1C09FF1FD2
:101FD0004A0AFF1F70B580241025E405A3682B432F
:101FE000A36001F0B9FFA368AB43A36070BD00001C
:101FF000F7B5160080221C001023D20501919168CC
:1020000005000B43936000225A4BD7301A6001F051
:102010006BFF9D232A002F009B00EB58CA32012141
:102020000092FC37002B01D00021009A386801F0A3
:1020300023FF2900009BCB311A784F4BD3351A6010
:102040004B780A781B0213438A7812041A43CB7820
:102050001B061343494A1BBA13604B790A791B02CA
:1020600013438A7912041A43CB7931001B061343B8
:10207000434A1BBA13606B782A781B021343AA7871
:1020800012041A43EB781B0613433E4A1BBA136033
:10209000019A330213433C4A13603C4B22001B1B42
:1020A0009C4603293DDCB3089A0013005142B21A42
:1020B000032A46D1354AE018511A82784078120432
:1020C00000020243E05C043302430A600022FF2B5B
:1020D0004BDDF0222E4B12011A600F222D4B1A609D
:1020E0002D4A1368002BFCD00023224A2749136095
:1020F000091B321D0B191B68043A180A2370607003
:10210000180C1B0EA070E3700434002AF2DC80224D
:1021100010213B68D20501333B6093688B43936089
:10212000F7BD6346D578981893782D061B042B438A
:10213000157804392B43557804322D022B43036064
:10214000AFE7022A0AD1114AE05C511AE21852782C
:10215000120202430A6004339BB2B7E7012AB5D1E9
:102160000A4A521AE15C1160F5E7084959180A60F9
:102170000433ACE7000004403C0004403800044055
:1021800034000440300004400C00044000010440CE
:10219000040004401000044014000440F7B515008A
:1021A00080221C001023D2050091916807000B4388
:1021B00093600023654AD730136001F095FE9D239C
:1021C0003E009B00F9583B00CA363200FC33002920
:1021D00000D07FE0586801F04FFE390032785C4B48
:1021E000CB311A604B780A781B0213438A78AC46CD
:1021F00012041A43CB78281D1B061343554A1BBAF9
:1022000013604B790A791B0213438A7912041A432B
:10221000CB791B061343504A1BBA13604B7A0A7AD8
:102220001B0213438A7A12041A43CB7A21001B063D
:1022300013434A4A1BBA1360009A2B021343484ABD
:1022400013602200474B1B1B0093009BCE785B184A
:1022500001938B7836061B0433430E7804383343DE
:102260004E78043136023343019E33600328ECDCA0
:102270000321A808431C9B002940800003292BD17F
:102280003849E5185E18A9786D78E35C09042D02D9
:10229000294319433160030008330021FF2B2DDD52
:1022A000314B324919600F21314B19600123274905
:1022B0000B60304B19680029FCD006211B680B40CD
:1022C000042B20D080220020D20593680A318B4352
:1022D0009360FEBD01217DE7022908D121495D18E7
:1022E000E1184978E35C090219432960D3E7012921
:1022F000D3D11C495918E35C0B60CCE71948181876
:1023000001600433CAE7002310490B606346002BC9
:102310000CDC3B00FC335A68102101325A608022E9
:10232000D205936801208B439360D2E7009B9B18F2
:102330001B68190A13705170190C1B0ED3700423FB
:102340005B4291709C440432E0E7C04600000440C8
:102350003C00044038000440340004403000044095
:102360000C0004400001044004000440080F000079
:10237000100004401400044070B5061E19D002225B
:10238000614B9B799343012B13D1604B1A78FF2A41
:102390000FD15A78FF2A0CD19A78FF2A09D1DA781E
:1023A000FF2A06D11A79FF2A03D15B79FF2B00D1CE
:1023B000A7E0574B0C201A78012A08D00022554D6F
:1023C0001A702B781A00093A042A01D8212070BD0E
:1023D0005A1F012AFAD94C4CA07B042800D990E05E
:1023E000A279032A00D98CE0821E012A03D86288D0
:1023F0001F2A00D885E0002E61D0012E00D080E099
:10240000A288012AE2D0002B0AD10138032803D880
:1024100001F0EEFC151D19151F202E7001F054FF60
:102420002B785A1E032A16D800253B4B1D60282303
:10243000237501F0F1FCA8422ED0A580C6E7022347
:1024400020202B70EAE7042322202B70E6E70323E9
:1024500021202B70E2E7073B012BB7D82F4B1B68DD
:10246000DB6A9B06B2D52E4B1A78002AAED1A27B2E
:10247000911E012901D9002AA8D1022280211A70B7
:102480002823284D89012878237501F0DDFD80215E
:102490002878890101F0A8FD0123A380224B1B7835
:1024A000002B0AD0FA228021204B92001B880902BF
:1024B0005A431C4B187801F0E7FC002087E701F035
:1024C00003FE2B78A680073B012B06D918482E70F7
:1024D00001F0E2FD1E2001F0F7FE114B114C1A78BD
:1024E000002A06D080210022207889011A7001F08C
:1024F000ABFD01F061FD80212078090201F0A4FD0F
:10250000DBE7122063E7C046A60BFF1F6B09FF1F26
:102510001A09FF1F1C09FF1F4809FF1F6C67FF1FD7
:102520002309FF1F1B09FF1F2109FF1F2C09FF1F84
:102530000010004010B5002901D001F0E5FE10BDEB
:10254000F7B5604B01919978A1239B004B435E4AFC
:10255000060014681022E418D6235B00E0583623E6
:10256000FF33E35C00279343222B41D1574B0F3AB3
:102570001A600760012501F007FD019B1880E82320
:102580005B00E35C002B01D0B34258DD0023504FC9
:10259000FB70AD33FF33E3581A68002A03D09B88E1
:1025A000DB439B071DD03823FF33E35C002B18D09F
:1025B0009B235B00E35C002B13D1D133FF33E35C3F
:1025C000B3420EDAA4235B00E15AE018090A023193
:1025D00001F04AFD23000122FE33013E01351A8736
:1025E000FA70E8235B00E35C002B2AD0A8B2FEBDA2
:1025F00003683D00002BBED081880430090A0231F7
:1026000001F032FDD6235B00E3581F60B2E72300E0
:10261000B133BA00FF339858013781880430090A72
:10262000023101F021FDE8235B00E35CBB42EEDCFC
:10263000E822F61AED1800235200A354A6E700275B
:10264000F1E7200001F0A0FD00281FD0002E1DDDC5
:102650007319882647190193B600200001F09CFDEC
:102660005A30800020184068013581880430090AFA
:10267000023101F0F9FC200001F066FDA35901339D
:10268000A351BD4202D0019B9D42E6D1114BE35CB8
:10269000002BABD095239B00E35C002BA6D00E4B08
:1026A000E15A0029A2D00D4AA35C994202D9013314
:1026B000A3549BE700231A212000A35401F01CFD22
:1026C00094E7C046300DFF1F3409FF1F001403407C
:1026D000E010FF1F5A020000720200005E020000BC
:1026E000F8B51D4B1D4F1A78002A10D1BA7B002A6D
:1026F00002D101321A7003E0032AFAD0022AF8D07C
:1027000001F08AFB00220120154B1A70F8BD154B11
:10271000154D1C68154B9E7801232B702878C0B28C
:1027200000F0CEFCBB7B002B0BD101F025FCA123DC
:102730009B007343E41883239B00E41823782B70D9
:10274000E4E7032B02D101F07FFDF0E70020022B2C
:10275000DCD101F071FCEAE71C09FF1FA60BFF1F8B
:102760002309FF1F3409FF1F490AFF1F300DFF1FF8
:10277000F0B587B00EAD2F780FAD2D780593AC4630
:10278000634614000E4D0CAA12782E7803930D9B0D
:10279000009201932200059B029701F04DFB2E70E1
:1027A000012C01D0042C08D1802206498B88934348
:1027B000054A1278D20113438B8007B0F0BDC046A2
:1027C0001C09FF1F6C11FF1F7809FF1F0B001B3B2B
:1027D00070B504003020E02B0DD81300E025493BF4
:1027E000FF3B9BB2ED00AB4205D8034B20001982A2
:1027F0005A8201F091FB70BD8410FF1F10B501F0EB
:102800009BFD054B00205B68052B04D9034A5268E9
:10281000D20200D4980810BD00100040FCE100E096
:1028200070B501F051FC0D4B1B68FC33DC691D6A6F
:10283000FFF7E4FF6419844204D2094B01241B68AA
:10284000002B07D004220024064B1A70064A936915
:102850000133936101F0B0FB200070BD6C67FF1F76
:102860009809FF1F2309FF1FFC0FFF1F70B50C4DB8
:102870002B68FC335C6A01F027FCFFF7BFFF2B6875
:102880000025FC339B6AE318834204D2054B1B6886
:10289000AB4200D1051B01F08FFB280070BDC04684
:1028A0006C67FF1F9809FF1FD722044B92009B58AB
:1028B00010B5002B00D0984710BDC0460000FF1F88
:1028C000F0B587B001F01EFAFFF7EEFFC54BC64C1E
:1028D00004931B78022B45D1C44B1B68186A01F086
:1028E00063FCC34BC34A1A60C34BC44A1A60A0229C
:1028F000C34B52001A60049B187801F0F5FCC149E3
:10290000C14801F0C1FCC149C14801F0BDFC102221
:10291000C04BFF201A60802252031A60802292036B
:102920001A60802212041A6001F0A6FB012001F057
:102930000BFBFA20400001F077FC582001F04CFC22
:10294000B54801F0B9FC012001F026FB072001F099
:10295000F3FAE26DB14B1A4084235B001343E36545
:1029600007B0F0BD01F058FCAD4E0290322001F0EE
:102970001BFC33681B0628D43C2001F015FC0F20FB
:1029800001F012FC974B1B78012B00D113E180253D
:1029900033682B4200D0A1E0636C03202B436364B7
:1029A00001F002FC01F038FC029B0299C31A5A1E86
:1029B000814200D81A009B4B1A608C4B19681E2369
:1029C0005343994A9B18CB618BE701F025FC802388
:1029D000E26BDB0213430390E363E26D8F4B032052
:1029E0001A4028231343E36501F0DEFB0320A56EA4
:1029F00001F0DAFBA36E0320DB03DB0B019301F094
:102A0000D3FBA76EED03FF03ED0BFF0B874AAB185B
:102A1000C22B2ED8019B9B18C22B2AD8BB18C22BC5
:102A200027D8019B2A009D4200D21A00019B9D429B
:102A300000D91D003B00974200D21300BD4200D9CF
:102A40003D005B1B122B14D80C22336814209343D7
:102A500033603368764A1340336001F0A5FB0821E8
:102A6000A36EE26DDB038A43E265724ADB0B1360FF
:102A700085E7032001F098FBA36EDB03DB0B0593D6
:102A800001F0CAFB039B0399C21A531E814200D86E
:102A90001300694A93421BD9FF23356864492D0A04
:102AA0001D4032686B1C1B060A401B0C134333602D
:102AB0000C23326800209A43083B1343336001F033
:102AC0000BFA5E485E4BA840984205DCFEF73AFFE1
:102AD000019D0197059F99E75A48F7E700235A4E51
:102AE00033608023226CDB0213432364636C032076
:102AF0002B43636401F058FB336801333360802358
:102B0000626C5B021343636405230193E26D434BE4
:102B100003201A404D4B1343E36501F045FB0821A8
:102B2000A26EE36D434F8B43E3653B6802394B4331
:102B3000D203D20B9A420CD89B1A3B2B0BD8E36DD5
:102B400043490B40E365636C0B406364414B1A607F
:102B500028E7D31AF1E7019B013BDBB20193002B7D
:102B6000D4D1E36D3A4A1340E365636C1340636468
:102B70003368042B07D9BFF34F8F374B374ADA60DE
:102B8000BFF34F8FFEE7636C0320AB43636401F038
:102B90000BFBE26D214B03201A4028231343E3650E
:102BA00001F002FB0822A36EDB03DB0B3B60E36D4D
:102BB0009343E3659AE70722E36B1340012B02D1AD
:102BC000002001F091FB264D264AAB6802201340FD
:102BD000AB6001F0E9FA8023AA685B001343AB60A5
:102BE000E0E6C0464A0AFF1F00F000406C67FF1F86
:102BF000000003400180063DBC0003403408000093
:102C0000A40003407102000014100040FFFF3F00C9
:102C10002810004000E100E03075000000FEFEFFDB
:102C2000C4F000405467FF1F7206000091FCFFFFD4
:102C3000FF00FFFF5C67FF1FE30C0000E88000005F
:102C40005F361E0060361E00C045FF1F28000100D1
:102C5000FFFFFEFF5867FF1F00ED00E00400FA05CC
:102C60003CF00040FFFEFFFF694E336888331B686D
:102C700083F3088801F058F900F018FC654B664AA8
:102C80001B68934207D0002001F026F90221634A15
:102C900013688B431360FFF713FE614B614C187888
:102CA000C0B201F0E9FA0023A3600233A3605E4BD7
:102CB0000120236001F078FA0323A36001F0ACFA4D
:102CC000040001F039FB050001F0A6FA574B18602B
:102CD00001F012FB564B1968621A531EA14200D232
:102CE00013008022D203934201D39B029B0A3268D5
:102CF000D16AC90700D478E04E491C0C09689BB220
:102D00004C4359432402090A641803274A49FC32F8
:102D100093680A6849489B1A494A4A4E12684A49C8
:102D20009B18414A34609A183B400193036892080B
:102D30009C46019B0A6063440360042B03D9013263
:102D40003B400A6003600B684049E418200001F032
:102D5000EBF93F4F3D493B68C3183B6020000193AE
:102D600001F062F83B4C206808183849206088421E
:102D700005D9019B01333B6001F056F8216001F059
:102D8000F3F8354B1B78002B0ED001F0D5FA3168E3
:102D9000324B4A1B1B6812189A4233D2591A4919EE
:102DA000091A2F4801F070FA2E4C237A002B0FD00D
:102DB00001F0C2FA3168E3684A1B1218934224D921
:102DC000591A4919091A284801F05EFA002323729A
:102DD000264B83F3088801F047F8022001F074FACB
:102DE000002001F079F801F097FADC019900023433
:102DF000641A5900641A09214B438033CB40A4085C
:102E0000E41882E7FA218900CBE71949DBE7C046DD
:102E10006C67FF1F0C0AFF1FB64121031000004022
:102E2000490AFF1F14100040C4090000100AFF1FC8
:102E3000340AFF1F380AFF1F200AFF1F280AFF1F3E
:102E40001C0AFF1F5067FF1F240AFF1F71020000AA
:102E50006008FF1F2C0AFF1F1C09FF1FE408FF1F4B
:102E600000100040740BFF1F3C10004000000020C9
:102E7000DC050000A022054B92009B5810B5002BEA
:102E800001D0984710BD01F0C7F8FBE70000FF1F15
:102E9000A122054B92009B5810B5002B01D09847FA
:102EA00010BD01F0B9F8FBE70000FF1FA222054B9F
:102EB00092009B5810B5002B01D0984710BD01F02F
:102EC000ABF8FBE70000FF1FA322054B92009B58C5
:102ED00010B5002B01D0984710BD01F09DF8FBE71D
:102EE0000000FF1FA422054B92009B5810B5002B39
:102EF00001D0984710BD01F08FF8FBE70000FF1FDD
:102F000070B501F019FA514B1860042001F0DCF99A
:102F100001F072F80400C30702D401F0CDF870BDCF
:102F200000224B4B1A604B4B1878013804282CD8E0
:102F300000F05EFF03231B1F2700200001F034F880
:102F40000128ECD0444C2378042B71D101F054F9C2
:102F5000002806D000F0A8FF582001F03DF9022318
:102F60002370032001F0B0F9D9E7200000F0ACFF96
:102F7000E6E7200001F0D8F9E2E7200000F09CFF2E
:102F8000DEE7200000F0C0FFDAE700F05DFF05009B
:102F9000012808D1314B1B78053B012B03D82000B9
:102FA000FFF768FFCEE72C4B1B78022B01D0052BD7
:102FB00020D1022D28D12A4B9B7BAB431CD1200072
:102FC000FFF766FF254B18780128BBD16405B9D4FB
:102FD000234925224B7B034205D1233A13405A4211
:102FE000534126331A000B7D9342ABD9322000F0B7
:102FF000EBFFA7E7022D07D1184B1B78052B11D14A
:103000002000FFF753FFDDE7012D0BD1012B03D18A
:103010002000FFF759FF95E7062B03D12000FFF7AB
:1030200061FF8FE7200000F0F7FF022D8AD1C9E78A
:10303000032B04D10B4B987C00F0CEFF91E7072BBC
:103040008FD1094B987B01F047F88AE79C09FF1F55
:103050009809FF1F9009FF1F2309FF1F1C09FF1F6D
:10306000A60BFF1FBC0BFF1FD40BFF1FFA210A4B3F
:103070000A4A49001A640A4A5A500A4A04395A50FC
:10308000094A08319A64094A5A50094A5C315A502F
:10309000084ADA667047C0460000FF1F7127FF1F0D
:1030A0006D28FF1F2128FF1F7923FF1FE126FF1F27
:1030B000011EFF1FD51DFF1F10B500F081FE10BDC2
:1030C0008023F7B59C46264B264F01932649274A75
:1030D000274D284C284B02281AD1604638600868D2
:1030E000264E304080263603304308600199097827
:1030F000002909D11660224A2A60224A2260E02271
:1031000019689143A03A1BE08021C9021160F2E7DF
:1031100066463E600F68194E3E408027FF023E43E0
:103120000E600199097800290DD1176001280ED190
:10313000154A2A60154A2260E02219689143C03A74
:103140000A431A60F7BD802189021160EEE7E02191
:103150000F4A02432A600F4A22601A688A43F0E746
:103160004B0AFF1FE0000340D800034090000340DB
:10317000000003405000034040000340FFFFE3FF16
:103180000280063D804508220180063D80660822B7
:103190000080069880550822F8B51E4B80261A68D4
:1031A000002014003440324232D11A681A4F3243A0
:1031B0001A6001223B68063093433B6000F0F4FF45
:1031C0000122164D2B681E432E603B680A261343CE
:1031D0003B608027BF00124B1B683B4211D1013E70
:1031E000F6B2FF2E09D17E220E4B1C682B68E40B31
:1031F0001440934323432B6005E0082000F0D4FFE4
:10320000E9E7002EEFD180222B68600893432B6002
:10321000F8BDC046C4F000405CF0004018F000402B
:1032200068F0004060F0004010B500F09DFF012103
:103230005820034A00F0D8FFFFF7AEFF10BDC0468C
:10324000600AFF1F10B578220021034800F094FFA8
:1032500001F002F8002010BD746AFF1F70B5040071
:1032600000F032FF00230C200B4A010059438D1857
:10327000515C00290DD0A14208D1012300246B70BC
:1032800000F0C2FE00F098FE200070BD01330A2B52
:10329000EBD11224F6E7C046746AFF1F70B5040034
:1032A00000F012FF002319001D000D4A10780028BD
:1032B00006D0A0420CD1557001310C320A29F5D14B
:1032C000002B0AD100F0C8FF00F076FE002070BD90
:1032D0005078461EB0411B18EEE700F095FEF3E76C
:1032E000746AFF1FF7B504000C20002384460E4DBE
:1032F000019267465F43E85D7E19A04212D0002824
:103300000BD10A4B9C4662461B7808331370019B15
:1033100070707C557160B360FEBD01330A2BE8D13B
:103320000320F9E70720F7E7746AFF1F706AFF1FA1
:103330008020F8B5484BC0051B68C1248360474B0B
:10334000FF251A68012313434361454BA4001A6803
:10335000444B40211A60444B1A68444B1A60444B5A
:103360001A59AA431A51C52292009E58AE433143BE
:10337000802699509F583F49F6010F403E439E508A
:103380009E5880273602360A3043985080201A59BA
:1033900000020A4002431A5104341A59364E3F04BF
:1033A000324080263A431A511A5936061202120A3E
:1033B00032431A5108341A5980260A4002431A51DE
:1033C000C32292009F58B446AF4337439F509F5843
:1033D000294E0F4007439F509F58374080263604A0
:1033E000374380269F509F5836063F023F0A374397
:1033F0009F50C0221F59AF433A431A511A59120223
:10340000120A1643C6221E5192009C58AC436546D0
:103410002C439C509C5800250C4020439850C720BA
:1034200080001A58154C1140C02212020A431A504B
:10343000134B1B78DB08AB4201DC0020F8BD23787E
:10344000002B06D0A368002B00D0984701350C3420
:10345000EEE71220F2E7C0465846FF1F5446FF1F12
:10346000B0F000406C6AFF1FB4F00040686AFF1FB4
:1034700000E100E0FF00FFFFFFFF00FF746AFF1F95
:10348000706AFF1F030010B51F2809D8072200200B
:103490001340072404490A78A24313430B7010BD5C
:1034A00000230620F5E7C046706AFF1F034A04495F
:1034B000136800200B4013607047C0461CF00040AA
:1034C000FFFFC1FF054B06491B780A6805485B07EB
:1034D00002401B0B134300200B607047706AFF1FF4
:1034E0001CF00040FFFFC1FF70B50C25FFF7EAFF9D
:1034F0000A4B1C780A4BE4086543ED18002C01D1F7
:10350000200070BD2B78002B06D06B68002B00D0FC
:103510009847013C0C3DF1E71220F2E7706AFF1F6B
:10352000686AFF1F07B50422074801A900F0ACF93B
:10353000019B013305D18023044ADB0411680B434E
:10354000136000200EBDC0461C18001114F000408E
:103550001FB5002102220B0001910091052000F00F
:1035600033FE02230B490A681A42FCD1202303933D
:10357000039B5A1E0392002BFAD1074A1368002BB3
:10358000FCDA0B246C442000012100F06DFE207851
:1035900004B010BD90C8004000C8004013B504003E
:1035A0000A4B0193019B002B01D1112016BDFFF79F
:1035B000CFFF23000340044205D0052000F0F4FDB6
:1035C000019B013BEDE71800F0E7C046FFFFFF0756
:1035D00007B500F079FD80220821D205936A019198
:1035E000002B01D10739916202210C4A1160019927
:1035F000481E01900029FAD1033111600531019173
:103600000199481E01900029FAD11160002B02D1C6
:103610008022D205936200F0CFFC07BD00C00040BD
:10362000F0B52D4C89B02378002B4FD1FEF76AF905
:1036300002232A4F03903A681A42FCD120230693B2
:10364000069B5A1E0692002BFAD1254E3368002B9A
:10365000FCDA0120FFF7A2FF011E02D0112009B001
:10366000F0BD030003220190009005AD9F2000F003
:10367000ABFD0321280000F0F7FD02233A681A424F
:10368000FCD120230793079B5A1E0792002BFAD1E7
:103690003368002BFCDA0120FFF780FF0028DDD122
:1036A0000398FEF743F9AA786B7811041B020B43C9
:1036B00029780B4363601300113B0A49052B07D897
:1036C00001239340A3600B60012323700020C6E711
:1036D00080231B03F6E7C0464046FF1F90C800400A
:1036E00000C800409808FF1F1E4B30B55A68187874
:1036F0001D4B85B0D31859424B4101210093002343
:1037000000F0FAFB194B1A4A02259A6300221A6547
:1037100010325A658022C4219D65164B1648D2028C
:10372000DA6789004258154B80241A4080231B0415
:1037300013434350642341200393E40500F006FA49
:10374000402000F003FA6562039D6B1E0393002D79
:10375000FAD103236362FFF73BFFA562FFF760FF27
:1037600005B030BD4C46FF1F95FFFEF700C8004076
:10377000050001FF04E100E000E100E0FFFF00FFC1
:10378000F0B585B00700FEF7BDF8022305002D4C0B
:1037900022681A42FCD120230093009B5A1E0092FB
:1037A000002BFAD1284E3368002BFCDA0120FFF7FA
:1037B000F5FE002803D01124200005B0F0BD234BF6
:1037C0002360022322681A42FCD120230193019B2B
:1037D0005A1E0192002BFAD13368002BFCDA01202B
:1037E000FFF7DCFE0028E6D1194B1F600223226898
:1037F0001A42FCD120230293029B5A1E0292002BF4
:10380000FAD13368002BFCDA0120FFF7C7FE00284D
:10381000D1D1104B2360022322681A42FCD120230D
:103820000393039B5A1E0392002BFAD13368002B9B
:10383000FCDA0120FFF7B2FE041EBCD12800FEF71F
:1038400075F8B9E790C8004000C8004001000006C4
:10385000A8C800400180000110B50020FFF790FFCC
:1038600010BD000010B5064B18705960FFF73CFF03
:1038700000211320034AFFF735FD002010BDC0468C
:103880004C46FF1FE936FF1FF0B5040085B00392D8
:103890000291FEF737F8882263035B0B52051A4347
:1038A0008023DB059D6A8023274F0092BA6800269B
:1038B00001901B039A420CD9F82326001B041E40DA
:1038C0001C4206D08022214B52025E6219680A43D4
:1038D0001A60002D0BD100F0F7FB02221C4B1A607E
:1038E0008023DB055A62013A9A6200F065FB0023EF
:1038F000039A934220D1002D0AD100F0E5FB144B2E
:1039000003221D608023DB055A629D6200F054FB98
:103910008023BA681B039A4208D9002E06D00022E1
:103920000A4B0C495A621A680A401A600198FDF75E
:10393000FDFF002005B0F0BD009A0299D218127860
:10394000CA540133D4E7C0464046FF1F00C80040B8
:1039500000C00040FFFFFEFFF0B587B00291039268
:103960000400FDF7CFFF019000F0AEFB802302259D
:103970000122234EDB0535605D629A6200F01CFB7C
:10398000204F3B682B42FCD120230493049B5A1EFA
:103990000492002BFAD11C4D2B68002BFCDA01207D
:1039A000FFF7FCFD002802D0112007B0F0BD200079
:1039B000039A029900F050FA022304003A681A426E
:1039C000FCD120230593059B5A1E0592002BFAD1AA
:1039D0002B68002BFCDA0120FFF7E0FD051EE3D188
:1039E00000F072FB80230322DB0535605A629D6282
:1039F00000F0E2FA0198FDF799FFE0B2D5E7C04682
:103A000000C0004090C8004000C80040F0B58024CD
:103A100089B00600FDF776FFE405A36A022503934B
:103A2000029000F051FB0123304F3D606562A362BC
:103A300000F0C2FA2E4C23682B42FCD120230593C0
:103A4000059B5A1E0592002BFAD12A4D2B68002B9C
:103A5000FCDA0120FFF7A2FD002803D0112420008A
:103A600009B0F0BD244B2360022322681A42FCD126
:103A700020230693069B5A1E0692002BFAD12B6830
:103A8000002BFCDA0120FFF789FD021EE6D11B4B5B
:103A900003211E60030001900090202000F094FBA1
:103AA000022322681A42FCD120230793079B5A1E47
:103AB0000792002BFAD12B68002BFCDA0320FFF7CA
:103AC0006DFD041ECAD100F0FFFA80230322DB053E
:103AD0003C605A629C6200F06FFA039B002B01D19C
:103AE000FFF776FD0298FDF721FFB8E700C0004020
:103AF00090C8004000C800400100000694C8004083
:103B000007B5000201910422000A01A9FFF724FF72
:103B10000EBD000073B5050005240B4AA3005B42EF
:103B20009B1819686B46DE1D300000F0ADFA0228C4
:103B300004D133782B55013CEFD276BD052CFCD057
:103B40000128FAD10230F8E7140900111F2807D81C
:103B5000012380228340D20591680B439360704714
:103B60003F2808D80123802220388340D20551699C
:103B70000B435361F3E75F28F1D8012380224038DB
:103B80008340D205116A0B431362E8E71F2807D868
:103B9000012280218240C9058B6893438B60704766
:103BA0003F2808D80122802120388240C9054B696E
:103BB00093434B61F3E75F28F1D80122802140381D
:103BC0008240C9050B6A93430B62E8E71F2810D8AF
:103BD00080230200DB05153A1968012A06D8202245
:103BE0009143196019680A431A60704701228240A4
:103BF000F6E73F2811D880230200DB05353AD96863
:103C0000032A06D810229143D960D9680A43DA60A2
:103C1000EBE7012220388240F5E75F28E5D8422310
:103C20008022181A413B8340D205516A9943516260
:103C3000516A0B435362D8E710B50400012813D131
:103C4000A022184992050B685B015B0913430B60C6
:103C5000154B164A19681140154A0A431A6040224A
:103C600019680A431A6010BD0028FCD101000A201F
:103C700000F0F2F921000B2000F0EEF9C0220A4B0F
:103C8000920019680A4340211A601A688A431A6030
:103C9000B022044912060B685B015B0913430B60F9
:103CA000E1E7C04614F000401CF000407F00FEFF3A
:103CB00080FD010072B6074A1368013313600422C5
:103CC000054B1A600023054A13608022D205536019
:103CD000FEE7C0467808FF1FC0F00040C4F0004077
:103CE000044B054A1A60054B1A600022044B1A6007
:103CF0007047C046140AFF1F841E0000380AFF1FC9
:103D0000C4F000400023034A1360034A1360034ACF
:103D10001360704754F0004040F1004044F100400F
:103D2000002310B5184C8AB0009301932378012B1F
:103D300027D06946012000F0AFFA002817D1009B78
:103D400012490293019B06AA0393114B02A81B6818
:103D50000493104B1B68059300F0FEF810220E49E7
:103D600006A800F051FA002804D1FF232370002098
:103D70000AB010BD0123094A074902A8237000F0C8
:103D8000EBF80120F4E7C0467067FF1F102900110F
:103D9000082900110C290011202900117467FF1F48
:103DA00013B501246946012000F076FA034B009414
:103DB0000193FFF7B5FF200016BDC046BB0B000006
:103DC00010B5FFF79FFFFFF7EBFF002802D0024B73
:103DD000984710BDFEE7C046E1A2000002B471465C
:103DE00049084900095649008E4402BC7047C04644
:103DF00002B4714649084900095C49008E4402BC7E
:103E00007047C04603B47146490840004900095A4A
:103E100049008E4403BC704701B40248844601BC8B
:103E2000604700BFA9D8000001B40248844601BC25
:103E3000604700BF090E000001B40248844601BC7F
:103E4000604700BF9D6A000001B40248844601BC7F
:103E5000604700BFDD0C010001B40248844601BC8C
:103E6000604700BF9573010001B40248844601BC5D
:103E7000604700BF7997000001B40248844601BC46
:103E8000604700BF2144000001B40248844601BCE1
:103E9000604700BF8B52010001B40248844601BC58
:103EA000604700BFE94C010001B40248844601BCF0
:103EB000604700BF6DF6000001B40248844601BCB3
:103EC000604700BFF535010001B40248844601BCDB
:103ED000604700BF0934010001B40248844601BCB8
:103EE000604700BF016C010001B40248844601BC78
:103EF000604700BF8944000001B40248844601BC09
:103F0000604700BFC56D010001B40248844601BC92
:103F1000604700BFF935010001B40248844601BC86
:103F2000604700BF116E000001B40248844601BC26
:103F3000604700BFC9A9000001B40248844601BC23
:103F4000604700BFF90D010001B40248844601BC7E
:103F5000604700BF6911010001B40248844601BCFA
:103F6000604700BFDD3F000001B40248844601BC49
:103F7000604700BFD544010001B40248844601BC3B
:103F8000604700BFE9F6000001B40248844601BC66
:103F9000604700BFCD0C010001B40248844601BC5B
:103FA000604700BFE512010001B40248844601BC2D
:103FB000604700BF0134010001B40248844601BCDF
:103FC000604700BF9DA9000001B40248844601BCBF
:103FD000604700BF6137010001B40248844601BC5C
:103FE000604700BF4DF9000001B40248844601BC9F
:103FF000604700BF0D52010001B40248844601BC75
:10400000604700BFBD0B010001B40248844601BCFB
:10401000604700BF21A9000001B40248844601BCEA
:10402000604700BFE917010001B40248844601BCA3
:10403000604700BF75B7001101B40248844601BC57
:10404000604700BF19FA000001B40248844601BC71
:10405000604700BFB352010001B40248844601BC6E
:10406000604700BFADA3001101B40248844601BC03
:10407000604700BFC115010001B40248844601BC7D
:10408000604700BFED6B010001B40248844601BCEB
:10409000604700BF9938001101B40248844601BC52
:1040A000604700BFC1A5000001B40248844601BCBE
:1040B000604700BFA1AF000001B40248844601BCC4
:1040C000604700BFDD0A010001B40248844601BC1C
:1040D000604700BF75A9000001B40248844601BCD6
:1040E000604700BFC1F7000001B40248844601BC2C
:1040F000604700BFF9ED000001B40248844601BCEE
:10410000604700BF53B9000001B40248844601BCB7
:10411000604700BF51B8000001B40248844601BCAA
:10412000604700BF85C1000001B40248844601BC5D
:10413000604700BF090E000001B40248844601BC7C
:10414000604700BFE90B010001B40248844601BC8E
:10415000604700BF5976010001B40248844601BCA3
:10416000604700BFF9A6000001B40248844601BCC4
:10417000604700BFED68010001B40248844601BCFD
:10418000604700BFB70E000001B40248844601BC7E
:10419000604700BF71B0000001B40248844601BC12
:1041A000604700BFD9B0000001B40248844601BC9A
:1041B000604700BF0189000001B40248844601BC89
:1041C000604700BF8937010001B40248844601BC42
:1041D000604700BF496D010001B40248844601BC3C
:1041E000604700BF7912010001B40248844601BC57
:1041F000604700BF0167010001B40248844601BC6A
:10420000604700BF01D7000001B40248844601BCEA
:10421000604700BFCD4C010001B40248844601BC98
:10422000604700BF156B010001B40248844601BC21
:10423000604700BF8512010001B40248844601BCFA
:10424000604700BF8D82000001B40248844601BC73
:10425000604700BF75F8000001B40248844601BC05
:10426000604700BFADAE000001B40248844601BC07
:10427000604700BF3D71010001B40248844601BCA3
:10428000604700BF8914010001B40248844601BCA4
:10429000604700BF2D6C010001B40248844601BC98
:1042A000604700BFE1AC000001B40248844601BC95
:1042B000604700BF6D0B010001B40248844601BC99
:1042C000604700BF8D11010001B40248844601BC63
:1042D000604700BF1907010001B40248844601BCD1
:1042E000604700BFBD5C010001B40248844601BCC8
:1042F000604700BFEDA5000001B40248844601BC40
:10430000604700BFC166010001B40248844601BC99
:10431000604700BFE9D4000001B40248844601BCF4
:10432000604700BF8552010001B40248844601BCC9
:10433000604700BF0534010001B40248844601BC57
:10434000604700BFC95C010001B40248844601BC5B
:08435000604700BFE9270000EF
:1043580002000000DAC00011010000008CBE00114C
:1043680002000000D6C00011010000009843FF1FA2
:104378000200000094BE001101000000B064FF1F9D
:1043880002000000D4C00011030000002464FF1FD5
:104398001200000002000000DAC000110100000055
:1043A800D4BE001102000000D6C0001101000000B8
:1043B800D1BE001102000000DEBE001103000000A3
:1043C8005F64FF1F02000000D4C00011030000005A
:1043D8007464FF1F02000000D6C000110100000035
:1043E800D0BE001102000000DCBE00110300000076
:1043F8003564FF1F02000000D4C000110300000054
:104408005664FF1F02000000DAC00011010000001E
:1044180014BF001102000000D6C000110100000006
:10442800E144FF1F0200000026BF00110100000048
:104438000FBF001102000000D6C0001101000000EB
:10444800E044FF1F0200000024BF0011010000002B
:104458007C64FF1F02000000D6C0001101000000AC
:10446800DF44FF1F0200000022BF0011010000000E
:10447800FFBE001102000000D6C0001101000000BC
:10448800DE44FF1F0200000020BF001101000000F1
:10449800FABE001102000000D6C0001101000000A1
:1044A800DD44FF1F020000001EBF001101000000D4
:1044B800F5BE001102000000D6C000110100000086
:1044C800DC44FF1F020000001CBF001101000000B7
:1044D800F0BE001102020202020200000000000009
:1044E8000D0C0000514D0011174D001168BF00114F
:1044F800900118001800FFFF0701020304050602D7
:10450800010600000000000000000000000000009C
:104518000000000000000000000000000000030090
:1045280002000000DAC0001101000000E8BF00111D
:1045380002000000D6C00011010000009845FF1FCE
:1045480002000000F2BF001101000000AA64FF1F72
:1045580002000000D4C00011030000001867FF1F0C
:1045680002000000D6C00011010000009845FF1F9E
:1045780002000000F0BF001101000000AC64FF1F42
:1045880002000000D4C00011030000001067FF1FE4
:10459800126C6C6C000000000058004015160000FA
:1045A8000001000000000111FFFF000050485936CB
:1045B80000000000000000000100000079BF0011A9
:1045C8000B000500F7000000B400002800280028B0
:1045D8003075A000A000A000A00000080008E001BD
:1045E800F000100010001000100010001000500023
:1045F8005000500010001000D0070000000000001C
:104608000F0001000500307507001000010081FF50
:1046180000000000FF000000957500119D73001157
:104628002D710011FFFF0100FF000000B19F001174
:104638002D9D0011459C00110000000000000000A5
:1046480000000800040000003B0001085902E001D6
:1046580088212800FF00000002000000DAC00011D5
:1046680001000000A0C1001102000000D6C0001126
:1046780001000000DD46FF1F02000000D2C000114B
:10468800010000002C6BFF1F02000000D6C00011C3
:1046980001000000DC46FF1F02000000D0C000112E
:1046A80001000000DA46FF1F02000000D6C000111A
:1046B80001000000D846FF1F02000000CEC0001114
:1046C80001000000D046FF1F1800180000009001EC
:1046D800020000030202000002000000DAC000111C
:1046E80001000000B4C1001102000000D6C0001192
:1046F800010000002047FF1F02000000CCC000118D
:10470800000000000000000002000000D4C00011FA
:0A471800030000004C6BFF1F20FFA0
:040000051FFF184180
:00000001FF
